:020000040800F2
:2000000000500020697E0008B17E0008B17E0008B17E0008B17E0008B17E0008000000006E
:20002000000000000000000000000000B17E0008B17E000800000000B17E000807660008A6
:20004000B17E0008B17E0008B17E0008B17E0008B17E0008B17E0008F9670008FF67000880
:20006000056800080B68000811680008B17E0008B17E0008B17E0008B17E0008B17E0008FC
:20008000B17E0008B17E0008B17E0008B17E0008B17E0008B17E0008B17E00081768000858
:2000A000B17E000859630008B17E00086D630008716300088563000899630008013100082C
:2000C0000D3100081931000825310008B17E0008B17E0008C5740008DD740008F9740008AD
:2000E0003F680008B17E0008B17E00080000000000000000000000000000000000000000E3
:2001000000000000000000005FF808F1034613F8012B002AFBD1181A0138704710B5054CE1
:20012000237833B9044B13B10448AFF300800123237010BD0801002000000000848C0008F2
:2001400008B5034B1BB103490348AFF3008008BD000000000C010020848C0008704790F9C5
:200160002C30002BBABF90F82900C00900207047024690F82C3013F040001CBF92F8290031
:20018000C0F380107047024690F82C3013F020001CBF92F82900C0F340107047024690F8FE
:2001A0002C3013F010001CBF92F82900C0F300107047024690F82C3013F008001CBF92F82C
:2001C0002900C0F3C0007047024690F82C3013F004001CBF92F82900C0F3800070470246D9
:2001E00090F82D3013F010001CBF92F82A00C0F300107047024690F82D3013F008001CBFEB
:2002000092F82A00C0F3C000704700000122014B1A707047C003002010B50446034B0449C3
:200220000360044807F0C7FC204610BD049500089C8C0008F406002010B50446FFF7ECFF47
:200240002046302106F009F9204610BD012A02D1016000207047022A05D0032AF9D0002A65
:20026000F7D10260F5E70B680360F2E703681847012A02D1016000207047022A05D0032A9B
:20028000F9D0002AF7D10260F5E70B680360F2E7036808681847836810B5044613B1032299
:2002A00001469847204610BDCBB2322B08D80E4A01F4E06152F823301943C0F8881070479D
:2002C00001F0C002C02A0CD1CF2B0AD8074B01F03F0253F82220044B01F4E06153F8223095
:2002E000EAE74FF0FF31E8E7649B0008249B0008CBB2322B08D80E4A01F4E06152F823303C
:200300001943C0F88410704701F0C002C02A0CD1CF2B0AD8074B01F03F0253F82220044BC8
:2003200001F4E06153F82230EAE74FF0FF31E8E7649B0008249B0008036810B51B6B04460D
:2003400098474A2808D10423237123682046D3F8E0309847012010BD0020FCE770B5067B76
:20036000044616B1FFF7E8FF70BD012303730369ABB1D0E905230B490B4807F01CFC2069E0
:2003800002F0BAF9D4E904512846FFF7B1FF2846A169FFF789FF3146284602F039FC20462A
:2003A000E0E700BFAC8C0008F406002038B52C2007F09EFE01280446084D0CD12B78012B1D
:2003C00003D00749074807F0E3FB00210E2007F055FE2C7038BD0121F8E700BFBC0300200D
:2003E000BA8C00087002002010B5064B42F210705C7907F071FD2146BDE81040082007F09E
:2004000071BD00BF2401002038B5074D6C79044484F3080442F2107007F05EFD2146082024
:2004200007F060FD6C7138BD2401002070B50E4A0E4913780E4E013303F00303CC5C1370BE
:20044000B27A42F210701444A4F11403EB2B254684BF00252C4607F03FFD2946282007F07C
:2004600041FDB47270BD00BF55020020000000202401002000212D2007F000BE01212D20BE
:2004800007F0FCBD70B505460C460026AE4205DB2146BDE870402D2007F0F0BDFFF7EAFF68
:2004A0004FF4C87007F064FEFFF7E8FFC82007F05FFE0136EAE700000022044B83F84020FB
:2004C00083F83F2083F83E20704700BF140200200F4982B0ADF8040091F83E001E2815D890
:2004E00091F84030BDF80420013021F813201F220133DBB2B3FBF2F281F83E000120C2EB94
:2005000042129B1A81F8403002B070470020FBE71402002007B5ADF804000198FFF7D8FF7D
:20052000D8B90F49BDF8042091F8403021F813201F220133DBB2B3FBF2F0C0EB40101B1AF2
:2005400081F8403091F83F300133DBB2B3FBF2F2C2EB42129B1A81F83F3003B05DF804FBC2
:200560001402002037B5144B1B7823B903B0BDE83040FFF7A1BF114C8DF80400A5788DF8E5
:200580000510EB0642BFE37843F00803E3700198FFF79EFF68B9AA0742BFE37843F00103D7
:2005A000E370EB0705D5019803B0BDE83040FFF7B1BF03B030BD00BFBD03002024010020D1
:2005C00037B5104A92F83E30D3B192F83F40013B611CC9B282F83F1012F8140002EB440400
:2005E00065781F24B1FBF4F482F83E302B46C4EB4414091B82F83F1040EA032003B030BD0D
:200600001846F9E71402002038B50024114B124DC3F8D440A3F8D840022115F8010B0134A7
:2006200007F0CEFC072CF7D100240C4D002115F8010B013407F0C4FC082CF7D10024084DE6
:20064000022115F8010B013407F0BAFC0C2CF7D138BD00BF34010020DC960008D496000887
:20066000C896000808B507F043FD003818BF012008BD0000D222064B00219A700A229A7184
:200680000522DA71FF2299725A71DA72704700BF240100202DE9F041D0F814E004460F4648
:2006A00016461D46BEF1000F04D0F446BDE8F041007C6047406818B94FF0FF30BDE8F081B9
:2006C000217C02F05BF86068394603681B689847606802F0D8F90028EED12A46217C6068DD
:2006E00002F0CEF960682A4603683146DB699847281A18BF4FF0FF30E0E7002307B58DF852
:2007000007300DF107020123FFF7C4FF431C18BF9DF8070003B05DF804FB10B51446FFF7D0
:20072000ECFF431C0ED0C117C4F12002A4F12003E04001FA02F2104321FA03F3184300F06C
:20074000010010BD0020FCE708B5032200210C30FFF7E3FF08BD10B500F10C0401210322DF
:200760002046FFF7DAFF014620B905222046FFF7D4FF10BD0020FCE708B5142931D8DFE834
:2007800001F00B11131517303030303030191C1E20222426282B2E00002280210C30FFF798
:2007A000BCFF08BD0122F8E70222F6E70322F4E70422F2E700229021F0E70122FBE70222E4
:2007C000F9E70322F7E70422F5E70522F3E70722F1E700229121E1E702221821DEE706224C
:2007E000E9E70020DDE7036810B59B680446984728B1A42104F10C00FFF77FFF10BD4FF0CA
:20080000FF30FBE708B501210C30FFF776FF4011431E5842584108BD08B501210C30FFF786
:200820006CFF4011831E5842584108BD38B500F10C05044648212846FFF75FFF492184F819
:2008400028002846FFF759FF4A2184F829002846FFF753FF94F8293094F828201B0284F89C
:200860002A0043EA0243C0B20021184338BD032108B50C30FFF741FFC0B208BD272108B56A
:200880000C30FFF73AFFC0F3810008BD08B527210C30FFF732FF431C0CBF002000F003004F
:2008A00008BD08B562210C30FFF727FF431C0CBF002000F01F0008BD642108B50C30FFF749
:2008C0001CFF00F0030008BD08B524210C30FFF714FF431C1FBF00F0070000EB800000EB74
:2008E000800080000CBF002000F6282008BD162108B50C30FFF701FF00F0070008BD08B56B
:20090000132972D8DFE801F00A18274547717171717171596567696B7375777982210C306E
:20092000FFF7EBFE00F01F0000EB800000EB8000800000F2DC5059E083210C30FFF7DDFE6B
:20094000431C52D000F07F031846462B4FEA8303184414DC0BE084210C30FFF7CEFE00F04C
:200960007F03462B18464FEA830204DC1044400000F5FA703AE0473B102B104402D8800010
:20098000C83804E000EB80008000A0F5E15080B22CE08521D1E786210C30FFF7AEFE411C44
:2009A00023D000F01F00192837D000EB800000EB8000800000F5AF6018E092210C30FFF7B6
:2009C0009CFE00F01F0000EB800000EB80008000CEE79321F2E79421F0E79521EEE7962108
:2009E0000C30FFF78AFE421CEBD1002008BD9721F6E79921F4E79A21F2E76A210C30FFF7C3
:200A00007CFE431CF1D000F0070000EB800000EB8000800000F62820E8E74FF49660E5E7DD
:200A200038B500F10C0500212846FFF766FE012104462846FFF761FE240204F4F85400F055
:200A40001F00204338BD38B5036805469B68984708B9002038BD0C3534212846FFF74DFE7F
:200A6000044635212846FFF748FE621CF1D0431CEFD0240204F4F854204380B2EAE773B5D7
:200A8000866904460D468DF8072036B10123007C0DF10702B04702B070BD4068B0B1217C14
:200AA00001F06CFE6068294603681B6898476068012203680DF107015B689847606801F020
:200AC000E2FF003818BF01204042E4E74FF0FF30E1E738B500F10C040D4620466921FFF75B
:200AE0000CFE431C0BD000F0C80242EA051242F005026921204602F0FD02FFF7C0FF38BDF1
:200B000008B5FFF7B7FCBDE8084001210148FFF7E0BF00BF8C03002010B51348FFF714FEEC
:200B200000B31148FFF75FFE04462D2007F0E0FA631E1F2B01460AD80120FFF7A3FC0A48F2
:200B4000FFF760FE70B1BDE81040FFF7D9BFA4F12103202B01D80220EFE7423C222CEED836
:200B60000320EAE710BD00BF8C030020504BF0B45C6805680173002C00F09880002D00F011
:200B80009580AE784B4A013E28789278042E2ED8DFE806F025031D21290052067FD4002845
:200BA00000F0848002290FD1A0F120035F2B0AD9A0F10803022B06D9D42804D000F14C035D
:200BC000DBB2032B6ED801212346F0BC18475306E5D5A22064E05706E1D5A32060E05606F3
:200BE000DDD5A4205CE05506D9D5A52058E0C12809D1012901BF93F8DB6083F8DA1086F0EF
:200C0000010683F8DB601206C9D593F8D72012B993F8D82032B1A0F14102192A01D96878DD
:200C2000BDE7012293F8DB501DB1A0F14105192D32D993F8D65015B993F8DD3023B301292A
:200C40000BD100F0FD032C2B30D020282ED042282CD0492828D1D120B6E703299FD12C28DD
:200C600004D16FF00900F0BCFFF7CEBB2E2801D10A20F8E7202804D04228EAD1F0BCFFF7F8
:200C80004BBFF0BCFFF7D2BB002A88D1A0F14103192B84D82030C0B2022995D193E7A12095
:200CA000022991D102218FE700288DD1F0BC7047340100202401002038B5037B04460D4683
:200CC000032B00F29480DFE803F002304158002900F08D8003689A78474B1AB101211A44DB
:200CE00082F8D41093F8DA1093F8D62089B1284693F8DC50002D4DD193F8D710002977D014
:200D00001AB140F20111A3F8DC10114600284AD04CE093F8D8000028EAD022B140F201111C
:200D2000A3F8DA10E3E71046E2E707F01FFA6368C01AB0F5967F05D902212046BDE8384052
:200D4000FFF714BF002D52D10321F6E70029FBD007F00CFA6368C01AB0F5967F47D907F012
:200D600005FAA368C01A642841D902212046FFF7FDFE07F0FBF9A06039E003689A7822B11B
:200D80001D4B1344002283F8D42000212160D4E7B1B90FE0A0B993F8D71021B9294693F8AE
:200DA000D8000028F4D00120A3F8DA0041B993F8D71011B993F8D81011B10121A3F8DC10C5
:200DC0001AB983F8DA2083F8DC201A6832B193F8DA0093F8DC1000B901B190470121204649
:200DE000FFF7C4FE07F0C2F900236060A36038BD0028DCD10146D2E734010020FF222DE94D
:200E0000F04F7D4B85B01A7007F0B0F97B4CD4F8D030C01A102840F2A8800026784B794DBE
:200E2000DFF8E491029303954FF0000BC846DA46029B012113F8017B3846029307F0C0F8B9
:200E40000021384607F01AF9704B0193019B13F8010B0193FFF706FC012380F0010111F0C4
:200E6000FF0103FA0BF200F083809E4209D1BBF1040F01BF604B93F800C02CF0100C83F8A3
:200E800000C02AEA020A4FF0000C5C4B9A68424500F0AC800CF1010CBCF10A0F03F1140300
:200EA000F4D140B9554A9168002972D001300A2802F11402F7D10BF1010BBBF1070F08F17A
:200EC0001808C3D1039B012103F801AB38460393013607F0D3F80021384607F071F8082EB5
:200EE00009F10309A0D14FF0000B4FF00109DFF82081484E404FDFF804A118F8010BFFF7BD
:200F0000B1FBBBF1070F80F00101C9B250D82B7800294AD003F07F032B70A4460023DCF877
:200F20000820B2425CD001330A2B0CF1140CF6D140B923469A68002A47D001300A2803F120
:200F40001403F7D10BF1010B5FFA8BFBBBF10C0F06F1030605F10105CFD1FF22294B1A7247
:200F600007F004F9254BC3F8D00005B0BDE8F08F012E09D1BBF1040F01BF1F4B93F800C06C
:200F80004CF0100C83F800C04AEA02025FFA82FA79E7142358432218117501210830C2F8AB
:200FA00008802044FFF788FE85E763F07F03B3E7ABF10802D2B23B7809FA02F219B123EA43
:200FC00002033B70A9E71343FBE7142301215843231808309E601A752044FFF76DFEB1E748
:200FE00058B2142303FB00A00830F6E7142303FB0C400830D6E700BF04000020340100204F
:20100000D49600085C02002020960008DC960008C8960008FC950008032910B5044602D993
:20102000042904D010BDBDE81040FFF752BD0C3469212046FFF761FB431CF3D000F0F9005B
:2010400040F0010269212046FFF719FDEAE770B504460D461646FFF750FB431C0CD00123D2
:2010600003FA06F2024329462046D2B2FFF707FDB0FA80F0400970BD0020FCE708B5002271
:2010800010210C30FFF7E3FF08BD000038B51348FFF75AFBB0B11148FFF7B4FB054688B9C8
:2010A0000E48FFF7A0FB1428044612DCFFF7E6F9012C08DC02210948FFF70BFD14B9074861
:2010C000FFF7DCFF38BD0321BDE838400348FFF700BDFFF7CFF92946F6E700BF8C03002093
:2010E00008B500210348FFF7F4FCBDE80840FFF7CDBF00BF8C03002008B5002268210C3060
:20110000FFF7A5FF08BD08B5022230210C30FFF79EFF08BD08B5002230210C30FFF797FFB2
:2011200008BD08B5032230210C30FFF790FF08BD08B5012230210C30FFF789FF08BD08B5C4
:20114000042230210C30FFF782FF08BD08B513292ED8DFE801F00A101214162D2D2D2D2DB2
:201160002D181B1D1F212325272A002280210C30FFF76DFF08BD0122F8E70222F6E70322CB
:20118000F4E70422F2E700229021F0E70122FBE70222F9E70322F7E70422F5E70522F3E7BC
:2011A0000722F1E700229121E1E702221821DEE70020DFE708B5002226210C30FFF747FFEC
:2011C00008BD70B50446002500F10C06FF2248213046FFF754FCFF224921304684F8285078
:2011E000FFF74DFCFF224A21304684F82950FFF746FC84F82A5070BD642238B5B1FBF2F558
:2012000002FB15139BB22BB11449154806F0D3FC002038BD40F62723994203D840F6282236
:201220001049F2E740F6E442914201D90E49ECE700F10C0424212046FFF75FFA431CE7D038
:2012400000F0F800A5F11A02024324212046D2B2FFF715FCB0FA80F04009DAE7CD8C0008F4
:20126000F4060020EF8C0008278D000870B504460D461646FFF741FA431C0DD0012303FA69
:2012800006F220EA020229462046D2B2FFF7F7FBB0FA80F0400970BD0020FCE708B5012294
:2012A00030210C30FFF7E2FF08BD08B5002230210C30FFF7DBFF08BD08B5042230210C3094
:2012C000FFF7D4FF08BD08B5032230210C30FFF7CDFF08BD08B5022230210C30FFF7C6FF61
:2012E00008BD08B5002268210C30FFF7BFFF08BD38B5036804465B6D0D46984728B12D4921
:201300002D4806F058FC002038BD142DFBD801A353F825F069130008771300087B13000835
:201320007F13000883130008071300080713000807130008071300080713000807130008A9
:20134000871300088D1300089113000895130008991300089D130008A1130008A5130008FF
:20136000AB130008B11300080022802104F10C00FFF77CFFC8E70122F7E70222F5E70322D1
:20138000F3E70422F1E700229021EFE70122FBE70222F9E70322F7E70422F5E70522F3E7BD
:2013A0000722F1E700229121E0E702221821DDE70622E9E75F8D0008F40600202DE9F84319
:2013C0000C460B462C49161E05462C4A2C4808BF0A462C4906F0EFFB14F0FF0710D005F140
:2013E0000C0740213846FFF788F9CEB344EA0002D2B23846402185F82B20FFF740FB07462A
:2014000014F47F4F13D005F10C08412140464FEA1429FFF772F936B349EA00095FFA89F251
:201420004121404685F82C20FFF729FB074314F47F0F10D005F10C0842214046240CFFF708
:201440005CF9A6B10443E2B24221404685F82D20FFF715FB0743B7FA87F04009BDE8F88371
:2014600020EA0402C4E720EA0902D2B2D8E720EA0402D2B2E8E700BFB08D0008A98D0008B4
:20148000F4060020B88D000808B511460022FFF795FF08BD08B511460122FFF78FFF08BDE0
:2014A00038B500F10C040D4620462721FFF725F9431C0CD000F0F30242EA850227212046A8
:2014C000D2B2FFF7DCFAB0FA80F0400938BD0020FCE738B500F10C040D4620462721FFF77C
:2014E0000CF9431C0BD000F0FC0045EA000227212046FFF7C4FAB0FA80F0400938BD0020B6
:20150000FCE7102938B50D4601D9002038BD00F10C0462212046FFF7F0F8431CF5D000F0A4
:20152000E00045EA000262212046FFF7A8FAB0FA80F04009EAE7052938B50D4601D900207D
:2015400038BD00F10C0464212046FFF7D6F8431CF5D000F0FC0045EA000264212046FFF7C4
:201560008EFAB0FA80F04009EAE738B500F10C050C4628461621FFF7C0F8431C0CD000F0F0
:20158000F80004F00702024316212846FFF777FAB0FA80F0400938BD0020FCE738B500F1CC
:2015A0000C050C4628468321FFF7A7F8431C11D0A4F5FA73B3F52F7F00F0800018D80A22F9
:2015C000B4FBF2F302FB1344A4B22CB11049114806F0F1FA002038BDA3F132020243832197
:2015E0002846D2B2FFF74BFAB0FA80F04009F2E7A4F2C443B3F5A07FECD81422B4FBF2F390
:2016000002FB1344A4B2002CE0D103F10A02E5E7C88D0008F406002038B500F10C050C46BF
:2016200028468421FFF769F8431C12D0A4F5FA739AB2B2F52F7F00F0800018D80A22B4FB1D
:20164000F2F102FB114189B229B11949194806F0B2FA002038BDB3FBF2F2024384212846DF
:20166000D2B2FFF70CFAB0FA80F04009F2E7A4F2C443B3F5A07F0AD81422B4FBF2F302FBA1
:201680001344A4B2002CE0D103F10A02E5E7A4F5C863B3F5E16FDCD86422B4FBF2F302FB6D
:2016A0001344A4B2002CD0D103F14802D5E700BFEA8D0008F406002038B500F10C050C461D
:2016C00028468521FFF719F8431C11D0A4F5FA73B3F52F7F00F0800018D80A22B4FBF2F333
:2016E00002FB1344A4B22CB11049114806F063FA002038BDA3F13202024385212846D2B2A4
:20170000FFF7BDF9B0FA80F04009F2E7A4F2C443B3F51B7FECD81422B4FBF2F302FB134420
:20172000A4B2002CE0D103F10A02E5E7EA8D0008F4060020642238B5B1FBF2F302FB1313EA
:201740009BB20C4623B11E491E4806F034FA0DE0B1F5966F12D0B1F5AF6F09D24FF4AF63B7
:201760004FF496621849174806F025FA002038BD40F67462914201D91449E5E700F10C0560
:2017800086212846FEF7B9FF431CEFD0B4F5966F1EBF6423A4F5AF64B4FBF3F400F0E00243
:2017A00018BF22434FF0860128460CBF42F01902D2B2FFF764F9B0FA80F04009D7E700BFEA
:2017C000CD8C0008F40600200B8E0008378E000870B56426B1FBF6F306FB13139BB20C4616
:2017E00033B132461549164806F0E5F9002070BDB1F5FA7F03D24FF4FA721249F3E740F6A2
:20180000AC52914201D91049EDE700F10C0596212846FEF772FF431CE8D0A4F5FA74B4FB96
:20182000F6F400F0E00044EA000296212846D2B2FFF725F9B0FA80F04009D8E7CD8C00087E
:20184000F40600205D8E00088D8E000870B56426B1FBF6F306FB13139BB20C4633B13246F2
:201860001449154806F0A7F9002070BDB1F5FA7F03D24FF4FA721149F3E740F64852914251
:2018800001D90F49EDE700F10C0599212846FEF734FFA4F5FA74B4FBF6F400F0E00020431D
:2018A000C2B299212846FFF7EAF8B0FA80F04009DBE700BFCD8C0008F4060020BD8E000802
:2018C000ED8E0008642238B5B1FBF2F502FB15139BB22BB11349144806F06DF9002038BD08
:2018E00040F62723994203D840F628220F49F2E740F6E4429142F9D800F10C046A2120460F
:20190000FEF7FBFE431CE9D000F0F800A5F11A0202436A212046D2B2FFF7B1F8B0FA80F0B4
:201920004009DCE71D8F0008F4060020558F0008036870B55B6D05460E461446984728B1D8
:201940009B499C4806F037F9002070BD142EFBD801A353F826F000BFAD190008FF19000885
:20196000091A0008131A00081D1A00084919000849190008491900084919000849190008B6
:2019800049190008271A0008711A0008B91A0008031B00084D1B00084D1B0008571B0008A6
:2019A000571B0008611B00086B1B00086421B4FBF1F301FB13439BB213B164227E4906E0ED
:2019C00040F2DB539C4206D840F2DC527B49794806F0F1F8B8E740F64852944201D9784947
:2019E000F5E7A4F2DC52B2FBF1F28221D2B205F10C00FFF744F8B0FA80F04009A5E7214606
:201A00002846FFF7CBFDA0E721462846FFF704FE9BE721462846FFF74FFE96E7214628465A
:201A2000FFF788FE91E76426B4FBF6F306FB13439BB2002BC1D1B4F5FA7F03D24FF4FA7289
:201A40006049C4E740F6AC52944201D95E49BEE70C3592212846FEF750FEA4F5FA74B4FBA7
:201A6000F6F4922100F0E0022243D2B22846C0E76426B4FBF6F306FB13439BB2002B9CD19B
:201A8000B4F5FA7F03D24FF4FA7250499FE740F6AC52944201D94E4999E70C359321284623
:201AA000FEF72BFEA4F5FA74B4FBF6F400F0E00222439321D2B2D9E76426B4FBF6F306FB16
:201AC00013439BB2002B7FF478AFB4F5FA7F03D24FF4FA723F497AE740F6AC52944201D92B
:201AE0003D4974E70C3594212846FEF706FEA4F5FA74B4FBF6F400F0E00222439421D2B298
:201B0000B4E76426B4FBF6F306FB13439BB2002B7FF453AFB4F5FA7F03D24FF4FA722F49A6
:201B200055E740F6AC52944201D92D494FE70C3595212846FEF7E1FDA4F5FA74B4FBF6F401
:201B400000F0E00222439521D2B28FE721462846FFF73EFEF9E621462846FFF777FEF4E69E
:201B600021462846FFF7AEFEEFE63222B4FBF2F602FB16439BB2002B7FF420AFB4F5FA7FFC
:201B800003D24FF4FA72174921E7B4F5AF6F03D94FF4AF6214491AE70C3598212846FEF7A7
:201BA000ACFD0A3E00F0E00232439821D2B25DE7A88F0008F4060020CD8C0008EE8F00082D
:201BC000159000083C9000086C9000089C900008CC900008FC9000082C9100085C9100089A
:201BE0008C910008BC910008ED9100082DE9F043012185B00D2006F0E3F900210D2006F002
:201C00003DFAFEF737FD784806224FF4E13105F02FFF764B76495A6E0024C1F884201B6EB2
:201C20007348C1F8883000231F211A4600F0F5FF42F210716E4800F087FD6E4B69460093F7
:201C40006D4B6B4803936D4B0194029300F09EFD6846FEF720FB6A4F6A4B6B4E69466448D6
:201C600001946A4C00930397029600F0BFFD6846FEF711FB94F80C80B8F1000F00F0908029
:201C80002046FEF759FB002840F0A1806049564805F07EFF00212C2006F092F901212D2006
:201CA00006F08EF900212D2006F0E8F901210E2006F086F901210E2006F0E0F942F21070CA
:201CC00006F00AF96421082006F00CF9FEF79CFC504B514A6FF0DE005A60FEF795FB012102
:201CE0000D2006F0CBF94FF42F614848FFF784FA4648FFF7D3FA4548FFF7FEF94348FFF7DA
:201D000002FA4248FFF706FA4048FFF70AFA04213E48FFF781F90221292006F051F90023DB
:201D200001933E4B6946032229200093CDE9026705F0E4FF6846FEF7AEFA4FF0FF32002301
:201D40003248FFF7A1FB3148FFF73BFA344A00232E48FFF79FFB1A213248FEF7CEFC421C5A
:201D600005D000F00F021A212E48FEF788FE1A212C48FEF7C2FC431C07D000F0F00040F0B9
:201D800001021A212748FEF77AFE0022264B1A600122264B1A7005B0BDE8F043FFF776B94C
:201DA00001231B214FF01A09214D23732846C4E905192561FEF79CFA49462846FEF774FAB3
:201DC0004146284600F024FF3423237758E70122184B0E481A70FEF74AFD17490246024837
:201DE00005F0E9FE56E700BF70020020649B0008A8040020CD20000891020008710200089B
:201E00006D020008BD2100084D0200088C0300201E92000834010020650500080D020008C9
:201E200000FC18009803002088030020BD030020C4030020BF0300203392000870B5164631
:201E40000546FEF75AFC044631462846FEF755FC621C07D0431C05D0240204F47C5420439D
:201E600080B270BD0020FCE7036810B5DB680446984728B13922382104F10C00FFF7DEFF03
:201E800010BD08B53B223A210C30FFF7D7FF08BD10B55A495A4805F061FE5A48FEF7B2FC90
:201EA000594C5A49002818BF2146554805F070FE5749534805F052FE5248FEF7ADFC534920
:201EC000002818BF21464E4805F062FE51494C4805F044FE01215048FEF70FFC4B4B4009B3
:201EE00014BF19462146464805F052FE4B49444805F034FE4348FEF72EFC4449002818BFF9
:201F000021463F4805F044FE45493D4805F026FE052200214048FEF700FC3C49002818BF2B
:201F20002146374805F034FE3E49354805F016FE01213948FEF7E1FB431C5DD000F0070090
:201F4000052808D8DFE800F003505254565836492B4805F01DFE3549294805F0FFFD2948C3
:201F6000FEF771FD0A220146254805F070FE3049234805F00DFE2F49214805F0EFFD2148AC
:201F8000FFF772FF0A2201461D4805F060FE28491B4805F0FDFD2849194805F0DFFD1948E8
:201FA000FFF76FFF0A220146154805F050FE2049134805F0EDFD1348FEF7C6FB78B11F4965
:201FC0000F4805F0CBFD0F48FEF70DFC0A2201460B4805F03CFE1A49094805F0D9FDBDE87F
:201FE0001040074805F0C2BD1649B1E71649AFE71649ADE71649ABE71649A9E7469200082F
:20200000700200208C0300203F92000843920008529200085F920008980300206A92000825
:20202000749200088092000892920008E1920008248D0008F1920008019300081393000843
:20204000269300089D920008A8920008B8920008C9920008D592000807B51A221B210F4897
:2020600000F0E4FA002205210D4B0E48C3E908221A739A600C4A19711A600C4A17211A61DC
:202080001622C3E9051234221A77332309220A21009305F09BFB03B05DF804FBC4030020A6
:2020A0008C0300207002002004950008A804002008B50448FEF7B0F8BDE80840024800F0A5
:2020C0002FBB00BF8C030020C403002037B5314800F086FA002829DD00242E4800F080FABA
:2020E00098B902229DF800302B4C2C4903F07F03043B207060700A70092B17D8DFE803F04F
:2021000028181616161016233644224800F06CFA04F108036B4403F8080C84F00104DCE7C0
:20212000FEF74EFAC0F307232370607003B030BD9DF801301A4D6B71FEF756F9052323707A
:202140006B796370F2E70B232370164B1B68F8E7154B93F8DD2093F8DB305B0143EA8213CF
:20216000124A92F83E2013432370DFE70C2323700F4B10481A68C4F801205A681B7A4260A0
:2021800003720A230B70D1E70D2323700A4B1B78D7E700BFA8040020660200206502002067
:2021A000240100205802002034010020140200205C0200206702002004000020024B034911
:2021C0001A78034800F0B4BB6502002066020020A804002010B50948FEF7B6FA68B10B23E6
:2021E000074C06482370FEF7FEFA0222054B60701A70BDE81040FFF7E1BF10BD8C030020E9
:202200006602002065020020A54B73B51B78002B00F0BA8105F0AAFFA24C2368C01A44F683
:20222000206398420ED905F0A1FF20609E48FEF7DAFA421C04469D4D9D4B40F0A7810022A2
:2022400028701A609B4B1A78002A00F099810022954C1A702046FEF7E9FA054696499748EC
:2022600005F07CFC10222946944805F0F2FC9449924805F073FC02222946904805F0F6FC24
:2022800094F92B30002B09DA94F92830002B05DA8C498A4805F07CFCFFF79CFF94F82B30CD
:2022A0005B0608D594F828305E0604D5FFF792FF7D48FEF7E3FE94F82B309D0607D594F8AB
:2022C0002830980603D580497C4805F061FC94F82B30190707D594F828301A0703D57B49CD
:2022E000764805F055FC94F82B309B0707D594F828309E0703D57649704805F049FC94F8D7
:202300002B30DD0707D594F82830D80703D571496A4805F03DFC6448FDF721FF18B16E492D
:20232000664805F035FC6048FDF722FF28B16B49624805F02DFCFEF7D3FE5B48FDF723FF38
:2023400080B15948FEF74FFA411C04BFFF230020564A18BFC3B21370554B6149186057483B
:2023600005F016FC5048FDF719FF58B1FF224F4B5C491A7000224E4B50481A6005F008FCF9
:20238000FEF7AEFE4848FDF714FF18B356494B4805F0FEFB5549494805F0E0FB04230025CF
:2023A000194653480DEB03020195FEF773F901AE0A2216F8011B414805F056FC01354D498E
:2023C0003E4805F0CBFB042DF2D13C4805F0CEFBFFF75EFD3448FDF7F7FE90B14649374881
:2023E00005F0D6FB00210D2005F048FE00210E2005F044FE2C480421FEF70EFE2A48FEF707
:202400003DFE94F82C309A0707D594F829309B0703D53A49294805F0BBFB94F82C30DE0751
:2024200007D594F82930DD0703D53549234805F0AFFB94F82D30580607D594F82A3059062F
:2024400003D530491D4805F0A3FB94F82D309A0607D594F82A309B0603D52B49174805F0A7
:2024600097FB1148FDF7BBFE104D78B10E48FEF7BAF90F4B20EAE070186020F08000234918
:2024800028700E4805F084FBFEF72AFE0648FDF7B1FE00284DD00448FEF7A5F938E000BFD1
:2024A000BF030020880300208C030020BE03002058020020C003002028930008700200204D
:2024C000379300083D930008519300085E9300087993000892930008AC930008B993000891
:2024E000C6930008D2930008DE930008F09300089803002007940008099400081A94000851
:202500002A9400083A9400084E94000865940008234B20EAE070186040F080002870214942
:20252000214805F035FB2148FEF70EF908B1FEF7E7FA94F82D305E0707D594F82A305D07A5
:2025400003D51B49184805F023FB94F82D30980707D594F82A30990703D51649124805F05C
:2025600017FB94F82D30DA0707D594F82A30DB0703D511490C4805F00BFB0C48FEF721FEF2
:202580000E4B1A780E4BDA7202B070BD18600748FEF738F944EAC0142C70FEF777FD51E6A1
:2025A0005802002075940008700200208C030020869400089E940008B2940008BE030020C4
:2025C0002401002008B5FFF71FFEFEF717FCFDF7EDFEBDE808400A2005F0CABD0020704795
:2025E000028BC08A101A70470346C28A018B914281BF0169885C0132DA8298BF4FF0FF304D
:202600007047028BC38A9A4286BF0269D05C4FF0FF307047806DD0F8DC302BB10023D43088
:2026200020F8B23CC36818477047000070B54FF47A730E460021C0E90113034615462B4AB3
:20264000044643F8C42BC0F8C4109C22C3E90111C0E93411C0E93611C0F8E010283005F02B
:2026600017FFF3B2322B19D8214A06F4E06652F823301E43EBB2322BC4F8846022D81C4AAE
:2026800005F4E06552F823301D4300232046C4F88850E36123842361A38270BD06F0C00269
:2026A000C02A0CD1CF2B0AD8124B06F03F0253F822200F4B06F4E06653F82230D9E74FF020
:2026C000FF36D7E705F0C002C02A0CD1CF2B0AD8084B05F03F0253F82220054B05F4E06509
:2026E00053F82230D0E74FF0FF35CEE7EC960008649B0008249B000838B50446283000F087
:2027000055FBE06918B105F05BFD0023E36100252069258410B105F053FD2561A58238BDA4
:2027200038B505460446074B45F8D43BFFF7E4FF2846FDF7B0FD04F1C400FDF7ACFD2046D5
:2027400038BD00BFEC96000838B5044600F12805284600F069FB94F8BE304BB928460549EA
:2027600000F062FC2846BDE83840034900F055BC38BD00BF1526000871280008012399409E
:2027800080F8243000238176438470470023F0B587B002AC02930593C4E901338B680546DC
:2027A0000E460BB3022220469847D6E9023794E80300CDE9000105F1C40292E8030084E8CB
:2027C0000300DDE9000182E80300D5F8CC20C5F8CC30D5F8D0302046C5F8D07004920593F2
:2027E000FDF759FD07B0F0BD1F46E0E70023F0B587B002AC02930593C4E901338B68054606
:202800000E460BB3022220469847D6E9023794E80300CDE9000105F1D40292E8030084E85A
:202820000300DDE9000182E80300D5F8DC20C5F8DC30D5F8E0302046C5F8E0700492059351
:20284000FDF729FD07B0F0BD1F46E0E738B5838A05468B420C4609D2202938BF20240069A2
:20286000214605F063FD10B12861AC8238BDFEE773B5846D0546D4F8CC30866EE3B1E28A2A
:20288000238B9A4218D331462046FFF7DFFF3246206905F1740105F04BFE0023E382D4F814
:2028A000CC30268301960BB906F0E8F9D4F8D03001A904F1C400984702B070BDB1F5806FBF
:2028C00070B505460C4610D8038C99420AD920290E4638BF2026C069314605F027FD18B1A5
:2028E000E8612E84204670BDFEE70024FAE713B590F8243004468DF807107BB1418C0131AB
:20290000FFF7DCFF40B10120638C9DF80710E269D154638C0133638402B010BD01220DF11F
:202920000701283000F0A8FAB0FA80F04009F3E770B590F8243004460E46154693B1418C5D
:202940001144FFF7BBFF10B90025284670BD638CE0692A461844314605F0EAFD638C2B4434
:202960006384F2E792B2283000F086FA0028EBD1EBE70346006918B100219A8A05F088BDDB
:2029800070470346C06918B100211A8C05F080BD704738B50446D1B94FF42A03A36594F8D0
:2029A000BE30012B16D1638CE269A17E04F1280000F0E2FA042828BF0420C5B22046FFF7CA
:2029C000E0FF0023638484F82430284638BD4FF02A43E3E70425F8E72DE9F04790F8BEA02A
:2029E0000446BAF1010F0F46154698469DF820609DF8249039D111467F00FFF727FFFFB239
:202A00007EB10023032E28BF032684F824A0A7766384013EF6B2FF2E1BD100212046FFF762
:202A2000B8FFB9F1000F1DD14FF42A03A36539462B46226904F1280000F038FA0023984209
:202A40002E461CBF1D462E462846E3822683BDE8F0872368F10028FA01F120461B68C9B2C4
:202A60009847D6E74FF02A43E0E70020EFE707B5019300230093FFF7AFFF03B05DF804FBA0
:202A80000123FFF7F4BF0121FFF783BF38B500250446C5820583FFF76CFF20466584FFF73E
:202AA00070FF38BDF8B50446D0F8840005F0C2F9002105F085FAD4F88420C2F30313042BC0
:202AC00048D8284D284E55F8233002F00F029B6856F82220DB4303EA12239BB2002B3FD0EE
:202AE000D4F8880005F0A6F9012105F069FA1F4BD4F888001B681E4CC0F30311B3FBF4F36D
:202B00000A24042904FB03F300F00F0225D8142756F82220174CC2F30F2255F821C0CCF861
:202B20001420D4F804E06668A6EB0E06B342FADCCCF81020D4F804C06668A6EB0C06B34289
:202B4000FADC013FE9D105F075F93946BDE8F84005F036BA00239B68FFDE00235B61FBE73D
:202B6000F8BD00BF0C000020309700082800002040420F00001000E02DE9F0410026044666
:202B8000C68206831F460D469046FFF7F2FE20466684A676FFF7F5FED4F8DC30C4F8804047
:202BA00033B104F1D401032208469847C4E93766002384F824306B0084F825306B1E5D4274
:202BC0005D41204684F8BE5084F8BF8084F8C07004F12805FFF766FF284694F825200949F2
:202BE00000F02CF894F8BE304BB92846064900F01BFA2846BDE8F041044900F00EBABDE893
:202C0000F08100BFA086010015260008712800080A4600230121FFF7AFBFC9B2FFF7ACBFA4
:202C2000162217210148FFF701BD00BFA80400200148FFF775BD00BFA8040020F7B50D46A1
:202C400017460446002800F09F805049C06D04F08DF84F490646206E04F088F80146002EFC
:202C600000F09280002800F08F80304604F0A5F82060002800F08880464B261D984260D1A5
:202C800003F5DE33DA6942F40012DA61DA6902F400120092009A1A6942F400121A611A6925
:202CA00022F400121A6142F21F03A4F864303A4B1E603749206E04F041F83449E06D04F0EF
:202CC0003DF8364B21689D4258D9354B9D4203D9344B9D4288BF00234FF480420025C4E9CB
:202CE00001134FF48043C4E9053594F8973002215B1B18BF01239B01236294F89830C4E9CA
:202D000003275B1B18BF0123DB0163622A4694F96400E56184F8415000F09EFA94F964004A
:202D200000F0CAFA2A46022194F9650000F094FA94F9650000F0C0FA304600F0AFFCF8B186
:202D4000FEE7194B9842B4D103F5DC33DA6942F48002DA61DA6902F480020192019A1A6922
:202D600042F480021A611A6922F480021A6142F22123A4F86430084B5E609AE70022ADE79A
:202D80000223A06684F8953003B0F0BDF49A0008C49A0008005400408C050020A0860100FF
:202DA000801A060040420F000058004010B5044690F9640000F08EFA94F9650000F08AFA70
:202DC000201D00F014FD0321206E03F0F7FE0321E06D03F0F3FE2368104A93420DD1104BD3
:202DE0001A6942F400121A611A6922F400121A61DA6922F40012DA6110BD0A4A9342FBD1FF
:202E0000074B1A6942F480021A611A6922F480021A61DA6922F48002EDE700BF0054004012
:202E20000010024000580040104B10B59942044606D90F4B994203D90E4B994288BF0023D5
:202E40006068026822F001020260A360074B201D994294BF002101218903E16000F01EFCEF
:202E60006268136843F00103136010BDA0860100801A060040420F00202A30B514D8002300
:202E80009CB2A24207D890F894301344DBB280F89430002030BD90F89440CD5C1C4404447B
:202EA00084F874500133EBE70120F3E72DE9F34705460F469046994600F0B6F9002406461D
:202EC000D5F830A004354B46424639462846CDF800A000F0B9FD022806D100F0A5F9841BDD
:202EE000642CF0D906201FE008BB00F09DF90646284601F01FFD202809D0632C07D800F0C5
:202F000093F9841B284601F018FD0028F0D0284601F013FD632C0CD882060AD443070AD4BA
:202F2000003818BF0120800002B0BDE8F0870420FAE70520F8E70320F6E710B56423044674
:202F4000043000F06DFC022810D0032806D090B194F84130202B18BF042004E094F8413074
:202F6000202B18BF052008BF022004E094F84130202B18BF062010BD2DE9F34704460E463D
:202F800091461F4600F050F980463FB901223146204602B0BDE8F047FFF7CFBF0025D4F8FB
:202FA00030A004343B464A4631462046CDF800A000F0E2FC022807D100F036F9A0EB08052F
:202FC000642DEFD906201FE008BB00F02DF90646204601F0AFFC202809D0632D07D800F0CC
:202FE00023F9851B204601F0A8FC0028F0D0204601F0A3FC632D0CD882060AD443070AD43A
:20300000003818BF0120800002B0BDE8F0870420FAE70520F8E70320F6E720B119B1C16667
:20302000043000F00DBE704720B119B10167043000F006BE704770B590F891300446012B64
:203040000D46A0F1040609D1436E3BB1836E30469847022384F89130002363668DB9E36EE0
:2030600084F891501BB1304684F890509847204694F8902004F170012023BDE8704000F0E6
:2030800069BD00230122636684F89120616E2046743131440423BDE8704000F096BD10B5FB
:2030A00090F891300446012B04D1436E13B1836E04389847022384F8913000232046636647
:2030C000BDE8104000F0BCBD436E1F2BDEBF436E0133436690F89130012BDAB205D1416EE6
:2030E00004237031014400F070BD7047002380F89030704790F892300BB900F0A1BD7047CA
:20310000014B186800F01CBF8C050020014B186801F070BB8C050020014B586800F010BF03
:203120008C050020014B586801F064BB8C0500200379012B07D10A2919D840F2C740C8402C
:2031400000F001007047022B0BD1022903D8081E18BF01207047063903298CBF00200120EC
:203160007047042B03D1142901D80248E7E70020704700BF1FF81900012303FA01F18368A3
:203180000B4383607047012303FA01F1836823EA0103836070478068C84000F00100704706
:2031A0007047000038B50E4B05461A784FF47A73B3FBF2F30B4A1068B0FBF3F000F09CF893
:2031C000044658B90F2D09D8024629464FF0FF3000F042F82046044B1D6038BD0120FCE7FD
:2031E000050000202800002008000020074A08B51368032043F01003136000F01BF80020B2
:20320000FFF7D0FFFFF7CCFF002008BD00200240034A044B11681B780B441360704700BF01
:203220009405002005000020014B1868704700BF9405002007490302CA6803F4E06322F4DE
:20324000E0621204120C134343F0BF6343F40033CB60704700ED00E0154B30B5DC68C4F3F4
:203260000224C4F10703251D042B28BF0423062D4FF0FF3594BF0024033C05FA03F321EA8E
:203280000303A54022EA0502A340002843EA0203ACBF00F16040074A4FEA0313DBB2ABBF60
:2032A00000F5614000F00F0080F80033135430BD00ED00E014ED00E0002807DB0123410954
:2032C000034A00F01F00834042F82130704700BF00E100E000280CDB01220649430900F050
:2032E0001F008240203341F82320BFF34F8FBFF36F8F704700E100E00138B0F1807F0BD2B0
:203300004FF0E023F021054A586182F823100020072298611A6170470120704700ED00E08C
:20332000002808DB01224309034900F01F008240603341F82320704700E100E0704708B5FB
:20334000FFF7FCFF08BD704710B5044650B1437903F0FF0213B90271FFF7F5FF01230020D3
:20336000637110BD0120FCE790F821200346022A06D0042282630120002283F820207047D4
:203380000268C06B116821F00E011160116821F00101116001211A6C01FA02F24260002038
:2033A00083F82110E8E7000008B590F82130022B03D004238363012008BD03681A6822F00A
:2033C0000E021A601A6822F001021A60174A93421FD0143293421ED0143293421DD01432D6
:2033E00093421DD0143293421DD01432934214BF4FF080734FF480130D4A5360012380F867
:203400002130002380F82030436B03B198470020D2E70123F0E71023EEE74FF48073EBE74B
:203420004FF48053E8E74FF48033E5E7080002400000024090F82100704700002DE9F74F9D
:2034400000244FF00F0E2646DFF884C1614B00F104080A6832FA06F502D103B0BDE8F08F78
:20346000012505FA06F702EA070537EA020276D14A68032A07D8013A022A00F28380DFE8E5
:2034800002F091969C00122A00F0948069D8112A00F08A80FF2D94BF8146C1464FEA8602B3
:2034A000D9F8007088BF203A0EFA02FA27EA0A0704FA02F21743C9F80070D1F8049019F021
:2034C000805F4CD0DCF8182026F0030742F00102CCF81820DCF8182007F1804702F00102D4
:2034E000019207F5803706F0030A019A4FEA8A0ABA680EFA0AFB22EA0B0B374A904260D047
:2035000002F5806290425ED002F5806290425CD002F58062904214BF0422032202FA0AF23A
:2035200042EA0B02BA609A6819F4801F14BF2A43AA439A60DA6819F4001F14BF2A43AA43C8
:20354000DA605A6819F4003F14BF2A43AA435A601A6819F4803F14BF2A43AA431A60013610
:2035600077E7DFF878904A450CD014D8A9F580194A4507D009F570294A4503D0A9F58019EA
:203580004A4587D18A68D2B1012A4FF008040CBF076147617EE7DFF848904A45F2D009F51B
:2035A0008039EDE7CC6875E7CC68043472E7CC6808346FE7CC680C346CE700246AE70424FF
:2035C00068E70022AAE70122A8E70222A6E700BF00100240000401400008014000002210B5
:2035E00000003110044A08B55169014202D0506103F0ECF808BD00BF000401402DE9F8460B
:2036000006460F4691461D464FEA114A3368BAF1010F39D15C6927EA0404A4B2B4FA84F481
:203620006409A14501D0002024E06A1CEFD0FFF7FBFD089BC01AA84201D8002DE6D1BAF140
:20364000010F336818D15B6927EA03039BB2B3FA83F35B099945D9D1002320220120336383
:2036600086F83D2086F83E30326C86F83C3042F020023264BDE8F8869B69DB43C3F34003D3
:2036800083F00103DBB2E5E79C69E443C4F3400484F00104E4B2C4E77047000070B5044653
:2036A00008B9012070BD90F83D3003F0FF021BB980F83C20FFF7F0FF242384F83D302368CA
:2036C0001A6822F001021A601A6842F400421A601A6822F400421A6001F090FB3F4B65683E
:2036E0009D4294BF3E4B3F4B98428CBF00230123002BD6D1394E3C4BB542B0FBF3F388BF6A
:203700004FF496762268516821F03F0141EA030182BF73434FF47A76B3FBF6F35160116AAA
:20372000013321F03F010B431362D169431E2B4821F44F41854221F0FF0132D86D00B3FB91
:20374000F5F340F6FC700133034242D0C3F30B031943D1611168D4E9073021F0C00103437D
:203760000B4313609168D4E9030321F40341034321F0FF010B439360D168D4E9053021F09F
:20378000FF0103430B43D3601368002043F0010313602023206484F83D30206384F83E0030
:2037A00080E7A06850B905EB4505B3FBF5F30133C3F30B037BB143F40043C9E7192068438F
:2037C000B3FBF0F30133C3F30B0323B143F44043BEE70423BCE70123BAE700BFA0860100B8
:2037E0007F841E00FF083D0040420F00704710B5044698B12423026880F83D30136823F0A0
:2038000001031360FFF7F2FF0020206484F83C0084F83D00206384F83E0010BD0120FCE727
:203820002DE9FF4704461F4689469246FFF7FCFC94F83D300546202B03D0022004B0BDE80B
:20384000F08700901923012220464949FFF7D6FE0028F2D194F83C30012BEED0012384F8D3
:203860003C30236800261A6809F0FE09D2075EBF1A6842F001021A601A6822F400621A600E
:20388000242384F83D303B4B2664E36222684FF001111368204643F4807313603B460022A7
:2038A0000095FFF7ABFE236838B11B680320DB0544BF4FF400732364C0E7C3F81090FFF7A2
:2038C000B3FC4FF0A0080546226853695269C3F34003C2F3802294F83D10A02901D01343ED
:2038E0001DD04FF02008206884F83D80436913F0020F036843F40073036025D000230393CD
:20390000436901220393836919490393039B204619230095FFF772FE88B101208EE7FFF75E
:2039200083FC401BB84200D80FB984F83D80226853695269C3F34003C2F38022CBE784F85B
:203940003D8084F83C0079E76FF48063012243610749192320460095FFF750FE0028DCD1E5
:203960000136564592D384F83D8084F83C00D4E7020010000000FFFFF7B5002504460095A4
:20398000019594F83D500898202D02D0022003B0F0BD25682E68B60503D4082801D0012858
:2039A0001BD146F2A817274E3668B6FBF7F619277E430196019E013E0196019E56B9202375
:2039C000266384F83D3084F83E60236C43F020032364DBE7AE69B707ECD494F83C60012E41
:2039E000D4D02E68F6075EBF2E6846F001062E602E6826F400662E60212684F83D601026D8
:203A000084F83E60002626646385638DE06261642385236B62620093009B112B05D1B0F51E
:203A20002A0F02D0B0F12A4F03D12B6843F480732B60002084F83C006B6843F4E0636B6055
:203A4000A5E700BF28000020F7B5002504460095019594F83D500898202D02D0022003B0E0
:203A6000F0BD25682E68B60503D4082801D001281BD146F2A817364E3668B6FBF7F61927D7
:203A80007E430196019E013E0196019E56B92023266384F83D3084F83E60236C43F02003F7
:203AA0002364DBE7AE69B707ECD494F83C60012ED4D0012684F83C602E68F6075EBF2E68A8
:203AC00046F001062E602E6826F400662E60222684F83D60102684F83E600026266463852E
:203AE000638DE06261642385236B62620093638D9BB2022B24D1202801D0102820D1009B06
:203B0000122B2B681DD14FF4407223F480632B602B6843F400632B60009B122B05D1B0F562
:203B20002A0F02D0B0F12A4F03D12B6843F480732B60002084F83C006B6813436B608EE703
:203B40002B6843F480634FF4E0622B60E4E700BF2800002037B5044690F83D0000F02800C3
:203B6000282830D100292CD0002A2AD094F83C00012828D025682868C0075EBF286840F001
:203B800001002860286820F400602860292084F83D00202084F83E00002020646285628D9A
:203BA000E36201906B6961620193AB6984F83C000193019B6B68228543F4E0636B6003B096
:203BC00030BD0120FBE70220F9E737B5044690F83D0000F02800282830D100292CD0002A40
:203BE0002AD094F83C00012828D025682868C0075EBF286840F001002860286820F4006094
:203C000028602A2084F83D00202084F83E00002020646285628DE36201906B6961620193A4
:203C2000AB6984F83C000193019B6B68228543F4E0636B6003B030BD0120FBE70220F9E724
:203C400090F83D30202B14D1282380F83D30036800201A68D2075EBF1A6842F001021A60DB
:203C60001A6842F480621A605A6842F440725A6070470220704770477047704790F83D2032
:203C800008B5036DD2B283B9C36C0268012B836C05D1DBB21361036D0233036508BDC3F324
:203CA00007231361036D0133F7E7036D012B03D1836C0268DBB2F4E7036D022B2FD1222ACA
:203CC00005D10268136843F480731360EAE7438D9BB263B1212A0AD1436A026813F8011B26
:203CE00011614362438D013B9BB24385D6E7438D9BB2002BD2D1212AD0D10268516821F4C0
:203D0000E0615160116841F4007111602022036380F83D2080F83E30FFF7AFFFBEE703680A
:203D20005A69120644BF00221A61B7E770477047002337B546F2A81101932C4B406A1B68C4
:203D400090F83D20B3FBF1F323214B4301930368D2B2019941BB016C41F020010164446B2E
:203D60000CB10021A162816B09B100258D621D6825F480651D600025458504B1656301B18A
:203D80004D63196821F00101196090F83D10602911D1202380F83D30002380F83E3003648E
:203DA000FFF7C5FF03B030BD01990139019119688905CED4D3E702F02802282A0ED119680A
:203DC00041F001011960196841F4806119600023036380F83D20FFF78DF9E3E7202380F8C8
:203DE0003D30002380F83E30F5E700BF2800002010B590F83D2090F83E300446102BD9B2BA
:203E0000D2B2036801D0402913D1222A11D1196821F400611960596811F4006106D1602A6F
:203E20001EBF202284F83D2084F83E100022226307E002F028012829EDD10022226384F8E5
:203E40003D105A6812F400624FD05A68606B22F400625A6090F82130012B374B2BD04363E5
:203E6000FFF7A2FA50B12268606B136823F001031360202384F83D30436B9847236C1907ED
:203E80001FBF2268536823F4E063536094F83D30226CDBB252070DD5282B0BD1274B2022C0
:203EA000E36200232046236384F83D2084F83E30FFF7F5F810BDA06B4363FFF775FA0028FD
:203EC000DCD023685A69510605D51A69636A1A70636A013363622268A06B136823F00103F0
:203EE0001360202384F83D30C6E794F83D10602915D1202184F83D1022645A69520605D5A9
:203F00001A69636A1A70636A0133636222682046136823F001031360FFF709FFAEE75A69B6
:203F2000500605D51A69636A1A70636A013363622046FFF7DFF8A1E7313D00080000FFFF82
:203F4000F0B5044603688FB05A68C66A90F83E0094F83D101028C5B2C9B202D0402D40F09E
:203F6000E5829F69586910F0010F07D1B6F52A0F02D0B6F12A4F51D10FB0F0BD96054DD508
:203F8000E26AB2F52A0F0CD10122E26294F83E20402A11D1226D52B9626C02F0FE021A61A6
:203FA000EAE7E26AB2F12A4FF0D10822EDE7626C42F00102D2B2F2E72269B2F5804F1AD1BD
:203FC00094F83D20212A626C11D102F0FE021A61626B0AB1926A2AB9A26B002ACCD0926A5A
:203FE000002AC9D05A6842F400625A60C4E742F00102D2B2EBE7226D32B9626CD21102F097
:20400000060242F0F002CAE7226D012AB4D1626CD21102F0060242F0F102C0E7060703D528
:20402000960501D5626CE4E7860740F1F080960540F1ED8094F83E10E26A256B94F83D0090
:20404000C9B2222840F0DB80206D40B9402906D100905A6900929B690093009B8CE7216D32
:2040600089B92069B0F5404F0DD101915A6901929A690192019A1A6842F480721A60236D96
:204080000133236578E7618D89B251B902915A6902929A690292029A1A6842F400721A6011
:2040A00019E0618D89B2012949D112F5803F1BD11A6822F480621A605A6812F400620CD0EE
:2040C0001A6822F480621A60002203925A6903929B690393039B0023D3E704925A690492D9
:2040E0009A690492049AD7E7082A1CD0202A1AD0122D0DD1012A16D11A6822F480621A6056
:20410000002205925A6905929B690593059BE2E7102AF1D8864941FA02F2D707ECD41A6866
:2041200042F48062EBE71A6822F480621A60002206925A6906929A690692069AACE7618DD0
:2041400089B2022938D1102A03D87A49D140CE0718D4196841F4006119600021079159693B
:204160000791996907910799196821F48061196059680D05AFD5202A1BD8072A0ED8012AA7
:20418000A9D111E0196841F4806119600021089159690891996908910899E9E7A2F10801E7
:2041A000654ACA40D00796D55A6842F480525A6091E712F5803FE3E7196841F48061196068
:2041C0005968090510D5202A16D8072A06D8012A0AD15A6842F480525A6005E0A2F10801D9
:2041E000554ACA40D207F4D4002209925A6909929B690993099B6EE712F5803FE8E700220A
:204200000A925A690A929B690A930A9BB4E67F0740F194805E6836053FF5AEAE070600F06A
:2042200004063ED550053CD5002E3DD194F83D20258D94F83E10D2B2E06AC9B2C5B9212A38
:2042400018D1082858D0202856D010F5803F53D05A6822F4E0625A6011232363002384F89B
:204260003E302023204684F83D30FFF704FD83E6212A05D040297FF47FAE222A7FF47CAECC
:20428000628D92B21AB95A6822F48062ADE694F83E20402A16D120460FB0BDE8F040FFF7A0
:2042A000EDBC002E3FF468AE97057FF565AE212939D1E16A94F83D20212A7FF45DAE628D7B
:2042C00092B24AB1626A12F8011B19616262638D013B9BB263854FE608290DD020290BD0A7
:2042E00011F5803F08D0596821F4E06159601123236384F83E20B4E75A68204622F4E062A2
:204300005A601A6842F400721A6000232022236384F83D2094F83E2084F83E30402AA4D1C8
:20432000FFF7ABFC28E6402D7FF426AEB3E700BFEBFFFEFF140001000101000159680E05F2
:204340003FF51AAE450600F0040140F18680500540F18380002940F0838094F83D20222AD0
:204360007FF40AAEE06A628D92B2032A14D91A69636A1A70636A01336362638D013B9BB262
:204380006385638D9BB2032B7FF4F6AD2268536823F480635360EFE5E56A022D3FF473AF1B
:2043A000012A3FF670AF0B9146F2A811794A1268B2FBF1F202EB82020B920B9A013A0B9299
:2043C0000B99D1B9226C204642F0200222645A6822F4E0625A601A69636A1A70636A013332
:2043E0006362638D013B9BB26385202384F83D3084F83E10FEF77EFEBEE51A6812F4007293
:20440000DBD1196821F480611960596821F4E06159601969636A1970636A01336362638DA2
:20442000013B9BB26385202384F83D3094F83E3084F83E20402B04D122632046FFF776FC78
:204440009AE5082801D0202801D1002300E0122320462363FFF710FC8EE500293FF48CAD94
:2044600092057FF589ADE26A608D616A80B2042809D15A6822F480625A601B690B70636A7F
:204480000133636223E7608D80B203280CD15868042A20F480605860EFD0022AEDD01A682E
:2044A00022F480621A60E8E7608D80B20228E4D1042A33D007D8012A07D0022A2ED0186801
:2044C00040F4007004E0102AF9D1186820F4806018601B690B70616A4B1C6362638D013B42
:2044E0009BB2638523681B694B70636A216801336362638D013B9BB263854B6823F4407390
:204500004B60202384F83D3094F83E30402B4FF0000384F83E3005D123638EE7186840F4AE
:204520008060D5E7082A90D0202A8DE7206C20B30025586987072FD596052DD5226C02B1DA
:204540009D6994F83D2002F02802282A18D15A682F0622F480625A604FF0000354BFE268CD
:20456000A269C5F3800181F001012046C9B284F83C3092B2FEF75FFDFEE49D695869D9E7BD
:2045800000220C9259690C919B6984F83C200C930C9BF1E428000020C60640F1B1809505F5
:2045A00040F1AE8094F83D505A68EDB222F4E0625A6000220D925A690D921A6842F0010236
:2045C0001A600D9A1A6822F480621A605A68100520D505F0F702222A4AD1A06B0268526876
:2045E00092B26285628D92B21AB1226C42F0040222645A6822F400625A60FEF71BFF01281A
:2046000008D0A06B794B4363FEF7CEFE10B1A06B436B9847638D9BB213B323685A6951078A
:2046200009D51A69636A1A70636A01336362638D013B9BB2638523685A69520609D51A6994
:20464000636A1A70636A01336362638D013B9BB26385638D9BB21BB1236C43F00403236483
:20466000236C13B320460FB0BDE8F040FFF7C0BB606B0268526892B26285628D92B21AB162
:20468000226C42F0040222645A6822F400625A60FEF7D0FE0128BDD0606B544B4363FEF75C
:2046A00083FE0028B6D0606BB2E72A2D06D123632823204684F83D30FEF706FD94F83D3028
:2046C000282B0CD14A4B2022E36200232046236384F83D2084F83E30FEF7E1FC4CE4236B2C
:2046E000222B02D0222D7FF447AC00232022236384F83D2084F83E302046FEF7E5FC3BE4DD
:2047000001F0F701212900F0040535D1070627D5560525D53DBB94F83D00628DC0B292B2A3
:20472000002A3FF429AC626A12F8015B1D616262628D013A92B26285628D92B2002A7FF4AE
:204740001BAC29287FF418AC5A68204622F480625A602823216384F83D30FEF7C7FC0BE4D1
:20476000002D3FF409AC95057FF506AC628D92B2002A3FF401ACA5E5400627D5510525D50B
:204780003DBB94F83D20618DD2B289B200293FF4F3AB1969636A1970636A01336362638D03
:2047A000013B9BB26385638D9BB2002B7FF4E4AB2A2A7FF4E1AB2268536823F480635360D9
:2047C00022232363282384F83D3095E7002D3FF4D3AB92057FF5D0AB628D92B2002A3FF46A
:2047E000CBAB1A69636A1A7049E600BF313D00080000FFFFF8B5036804465F695E6890F88F
:204800003E2017F48075D2B20AD016F4807507D06FF4807101255961196841F40041196062
:20482000B80506D5F10542BF6FF4007145F002055961780536D5F10534D5608D94F83D10D2
:20484000202AD4F830C080B2C9B25FD100285DD101F0F700212804D0282957D1BCF1210FC4
:2048600054D194F83D20E16AD2B2082901D020292AD1282A28D12E4A2046E2625A6822F4D0
:20488000E0625A606FF480625A611A6822F480621A6000232022236384F83D2084F83E307A
:2048A000FEF7FDFB3A053FD5F3053DD56FF40062236845F008055A61236C20461D43256483
:2048C000BDE8F840FFF794BA212A1BD11849E16222630021202284F83D2084F83E105A688F
:2048E00022F4E0625A606FF480625A611A6822F480621A605A69100648BF19612046FEF7FD
:20490000F5FBCFE76FF480625A61CBE76FF48061102A596145F0040501D0402AC2D11A6879
:2049200042F400721A60BDE7002DC5D1F8BD00BF0000FFFF90F83D007047006C70470000DD
:204940002DE9F341054638B30368DB0710D42B689F075ED42B68190700F195802B685A078E
:2049600000F1C180EB69002B40F02C81002029E0904C636803F00C03042B07D0636803F013
:204980000C03082B0AD16368DE0307D523689C03DDD56B68002BDAD1012013E06B68B3F55E
:2049A000803F12D1236843F480332360FEF73CFC064623689803CAD4FEF736FC801B6428D2
:2049C000F7D9032002B0BDE8F0819BB9236823F480332360236823F480232360FEF724FC13
:2049E000064623689903B2D5FEF71EFC801B6428F7D9E6E7B3F5A02F236803D143F480233A
:204A00002360CFE723F480332360236823F48023CBE7684C636813F00C0F07D0636803F0E7
:204A20000C03082B10D16368DA030DD423689B0702D52B69012BAFD123686A6923F0F8031A
:204A400043EAC203236085E72A695B4B6AB101221A60FEF7E9FB064623689F07ECD4FEF779
:204A6000E3FB801B0228F7D9ABE71A60FEF7DCFB0646236898077FF56DAFFEF7D5FB801B85
:204A80000228F6D99DE7AA694A4E4B4BE2B10122C3F88024FEF7C8FB0446736A9B070DD5E0
:204AA0004FF4FA52454B1B68B3FBF2F3019300BF019B5A1E0192002BF9D14FE7FEF7B4FBF8
:204AC000001B0228E9D97CE7C3F88024FEF7ACFB0446736A9F077FF541AFFEF7A5FB001B90
:204AE0000228F6D96DE7334CE369D80024D40127E36943F08053E361E36903F0805300936B
:204B0000009B2F4E3368D90518D5EB68012B26D1236A43F001032362FEF786FB41F28838EF
:204B20000646236A9B073FD5002F3FF41BAFE36923F08053E36115E70027E2E7336843F486
:204B400080733360FEF770FB80463368DA05DCD4FEF76AFBA0EB08006428F6D931E7ABB9BB
:204B6000236A41F2883823F001032362236A23F004032362FEF758FB0646236A9807D3D585
:204B8000FEF752FB801B4045F7D91AE7052B236A03D143F004032362BAE723F00103236255
:204BA000236A23F00403B6E7FEF73EFB801B4045B7D906E7001002400000424228000020C8
:204BC000007000402A4C626802F00C02082A3ED00022022B274B1A662CD1FEF725FB064606
:204BE0002368990120D42B6AB3F5803F05D16268A96822F400320A436260696A62680B43AD
:204C000022F474121343012263601A4B1A66FEF70BFB054623689A013FF5A8AEFEF704FBED
:204C2000401B0228F6D9CCE6FEF7FEFA801B0228D6D9C6E6FEF7F8FA054623689B017FF594
:204C400095AEFEF7F1FA401B0228F6D9B9E6012B3FF4A2AE60682B6A00F480329A427FF43D
:204C60009BAE6B6A00F47010C01A18BF0120A9E600100240000042420D4A536803F00C0159
:204C8000082912D10B48C3F38341DB03405C09D55368094AC3F340435043084AD35CB0FBD5
:204CA000F3F07047064B584370470348704700BF001002401297000800127A0010970008B8
:204CC00000093D002DE9F0410D46044610B90120BDE8F081444A136803F007038B4228D3DC
:204CE00021688E0730D4CA0743D43F4A136803F00703AB4265D822683C4D12F0040F6CD11A
:204D0000130706D56B68226923F4605343EAC2036B60FFF7B1FF6B68354AC3F30313D35CC6
:204D2000D840344B1860344B1868FEF73BFA0020CEE7136823F007030B431360136803F09F
:204D400007038B42C3D1CBE7284B11F0040F1EBF5A6842F4E0625A60080742BF5A6842F4D6
:204D600060525A605A68A06822F0F00202435A60B9E762681D4E012A33681AD113F4003F2E
:204D8000A5D0736841F2883823F0030313437360FEF74AFA07467368626803F00C03B3EBC3
:204DA000820FA2D0FEF740FAC01B4045F3D903208EE7022A02D113F0007FE1E713F0020FA0
:204DC000DEE7136823F007032B431360136803F00703AB427FF47BAF8DE76B68E16823F4EC
:204DE000E0630B436B608BE70020024000100240789700082800002008000020044B054A0C
:204E00005B68C3F30223D35C034A1068D8407047001002407097000828000020044B054AEA
:204E20005B68C3F3C223D35C034A1068D84070470010024070970008280000200F23036013
:204E40000B4B5A6802F0030242605A6802F0F00282605A6802F4E062C2605B68DB0803F460
:204E6000E0630361034B1B6803F007030B6070470010024000200240036A026A70B522F0D7
:204E800001020262446882690D6822F073022A438D6823F002032B430A4DA8420BD1CD68DE
:204EA00023F008032B4324F44074D1E90556354323F004032C43446082614A684263036241
:204EC00070BD00BF002C0140036A026A70B522F4807202624468C2690D6822F073022A43CF
:204EE0008D6823F4007343EA05230B4DA8420DD1CD6823F4006343EA052324F44054D1E954
:204F00000556354323F4806344EA05144460C2614A68C263036270BD002C0140036A026A07
:204F200030B522F4805202624468C2690D6822F4E64242EA05228D6823F4005343EA05339F
:204F4000064DA84202BF4D6924F4804444EA85144460C2614A680264036230BD002C01405C
:204F600090F83D30012B1CD102230F4A80F83D30036893420AD0B3F1804F07D0A2F59432FF
:204F8000934203D002F58062934204D19A6802F00702062A03D01A6842F001021A60002095
:204FA00070470120704700BF002C014090F83C200346012A4FF0020009D01A6883F83D008A
:204FC00051610020012283F83C0083F83D20704770477047036870B5DD681E690446B107CA
:204FE0000DD5AA070BD56FF002021A61012202779B699B0769D001F02CFA00232377710799
:2050000010D56A070ED56FF00402236820461A61022222779B6913F4407F5CD001F019FACF
:205020000023237733070FD528070DD56FF00802236820461A6104222277DB69990750D0EC
:2050400001F007FA00232377F20610D5EB060ED56FF01002236820461A6108222277DB690C
:2050600013F4407F43D001F0F4F900232377F00708D5E90706D56FF00102236820461A614F
:2050800001F0C4F9320608D52B0606D56FF08002236820461A6100F004FB700608D5690643
:2050A00006D56FF04002236820461A61FFF791FFB20622D5AB0620D56FF0200223682046BB
:2050C000BDE870401A6100F0EBBA01F0C0F92046FFF77EFF91E701F0BAF92046FFF778FFF9
:2050E0009EE701F0B4F92046FFF772FFAAE701F0AEF92046FFF76CFFB7E770BD174A036839
:2051000090420AD0B0F1804F07D0A2F59432904203D002F58062904207D14A6823F07003DF
:205120001343CA6823F4407313434A6923F08003134303608B68C3620B688362074B984229
:2051400004BF0B690363012343610369DB0742BF036923F001030361704700BF002C0140D1
:2051600010B5044630B390F83D3003F0FF021BB980F83C2001F006FF0223206884F83D3020
:20518000211DFFF7BBFF0123002084F8463084F83E3084F83F3084F8403084F8413084F8C1
:2051A000423084F8433084F8443084F8453084F83D3010BD0120FCE7036A026A70B522F0E3
:2051C00010020262446882690D6822F4E64242EA05228D6823F0200343EA05130B4DA8420A
:2051E0000DD1CD6823F0800343EA051324F44064D1E90556354323F0400344EA85044460C7
:2052000082614A688263036270BD00BF002C014010B590F83C300446012B1DD0082A17D021
:2052200007D862B1042A0FD00120002384F83C3010BD0C2AF8D10068FFF770FE02E0006861
:20524000FFF71AFE0020F0E70068FFF7B5FFF9E70068FFF739FEF5E70220E9E738B590F87F
:205260003C300446012B4FD00120082A84F83C003AD006D8BAB1042A26D0002384F83C30A0
:2052800038BD0C2AF9D12068FFF748FEC3690A6943F40063C361C36923F48063C361C36982
:2052A00043EA02232EE02068FFF7E6FD83690A6943F008038361836923F0040383618369D6
:2052C000134383610020D8E72068FFF775FF83690A6943F400638361836923F4806383611C
:2052E000836943EA0223ECE72068FFF7EDFDC3690A6943F00803C361C36923F00403C361CA
:20530000C3691343C361DDE70220B9E770B5056A046A114E24F001040462B042846916D0BC
:20532000B0F1804F13D0A6F59436B0420FD006F58066B0420BD044F0010263F3071201F09F
:205340000A0125F00A0319438261016270BD24F003042243F1E700BF002C0140F8B590F898
:205360003C300546012B0C4600F081800120082A85F83C005BD006D842B3042A35D00023A7
:2053800085F83C30F8BD0C2AF9D1D1E900272B68CE68186A196A120321F480511962D96908
:2053A00020F4005021F4407141EA072102F4005266F30F310243D9611A62DA69A16822F432
:2053C0004062DA61DA6942EA01224EE02868CB6806C9FFF79BFF8369A26823F00C03836112
:2053E0008369134383610020C9E72B68D1E90027186ACE68196A120121F010011962996956
:2054000020F0A00021F4407141EA072102F0A00266F30F31024399611A629A69A16822F4B9
:2054200040629A619A6942EA01229A61DBE72B68D1E90021186A1E6AE76826F480761E6269
:20544000DE69120226F00306314320F4007002F4007267F307110243D9611A62DA69A168B9
:2054600022F00C02DA61DA690A43DA61BBE7022088E710B50124036A01F01F018C4023EA92
:2054800004030362036A8A401A43026210BD000008B529B990F83E30012B1DD001202EE0FE
:2054A000042907D190F83F30012BF7D1022380F83F3014E0082907D190F84030012BEDD111
:2054C000022380F840300AE090F84130012BE5D1022380F8413002E0022380F83E30006897
:2054E0000122FFF7C6FF0F4B984209D0B0F1804F0BD1836803F00703062B0DD1002008BD99
:20550000436C43F400434364F3E7074B9842F0D003F580639842ECD0036843F0010303607F
:20552000ECE700BF002C014000040040FFF7B0BF08B5034641BB90F83E0093F84220C0B29C
:205540000128D2B24DD1012A1DD1022291BB83F83E2083F8422018680122FFF78AFF224BB2
:2055600098420AD0B0F1804F07D0A3F59433984203D003F5806398422ED1836803F0070388
:20558000062B29D1002008BD042905D190F83F0093F84320C0B2D3E708290BBF90F8400054
:2055A00093F8410093F8442093F845200CBFC0B2C0B2C5E7042904D183F83F2083F843202B
:2055C000C9E708290BBF83F8402083F8412083F8442083F84520BEE7036843F00103036000
:2055E000D0E70120CFE700BF002C014010B50424036A01F00F018C4023EA04030362036AE4
:205600008A401A43026210BD08B529B990F84230012B1DD001203EE0042907D190F8433041
:20562000012BF7D1022380F8433014E0082907D190F84430012BEDD1022380F844300AE088
:2056400090F84530012BE5D1022380F8453002E0022380F8423000680422FFF7C7FF436C6F
:2056600043F4004343640C4B98420AD0B0F1804F07D0A3F59433984203D003F580639842F6
:2056800004D1836803F00703062B03D0036843F001030360002008BD002C0140FFF7B4BF89
:2056A00070477047026802F10C0353E8003F23F490730C3242E8003102680029F2D102F19A
:2056C000140353E8003F23F0010302F1140C4CE800310029F3D1036B012B0BD102F10C0345
:2056E00053E8003F23F0100302F10C0C4CE800310029F3D1202380F8423000230363704740
:2057000010B504460368C1681A6922F440520A431A6182680069D9680243606921F4B0513B
:2057200021F00C0102430A43DA605A69A16922F440720A435A610E4A934215D1FFF76EFB70
:2057400019234343626820689200B3FBF2F36422B3FBF2F102FB11331B013233B3FBF2F3A4
:2057600003EB0113836010BDFFF748FBE8E700BF00380140F7B505460C4617461E462A689B
:20578000136834EA030301D1002021E0701CF7D0FDF74AFDC01B86421CD3DEB12B68DA68F3
:2057A0005107ECD5802CEAD0402CE8D01A681207E5D5002401941A68284601925B6801935E
:2057C000019BFFF76FFF082301206B6485F8404003B0F0BD0320FBE7704710B5044648B38B
:2057E00090F8413003F0FF021BB980F84020FFF7F3FF2423226884F84130D368204623F4B2
:205800000053D360FFF77CFF236800201A6922F490421A615A6922F02A025A61DA6842F4CC
:205820000052DA602023606484F8413084F84230606310BD0120FCE710B5044668B390F8B4
:20584000413003F0FF021BB980F84020FFF7C4FF2423226884F84130D368204623F40053B5
:20586000D360FFF74DFF236800201A6922F490421A615A6922F022025A615A6942F008026F
:205880005A61DA6842F40052DA602023606484F8413084F84230606310BD0120FCE72DE9BD
:2058A000F843984690F841300446202B0E4617463FD100293FD0002A3DD0212300254564FF
:2058C00080F84130FDF7B0FCA3688146B3F5805FA784E78403D123690BB935461E46E38CDE
:2058E0009BB253B943464A4640212046FFF742FF202350B984F841300AE043464A4680215B
:205900002046FFF737FF28B12023032084F84130BDE8F88322684EB935F8023BC3F30803ED
:205920005360E18C013989B2E184D8E716F8013BF6E70220ECE70120EAE790F84130202B5C
:2059400010D189B182B1C28482840023212201620168436480F84120CA68184642F08002B7
:20596000CA607047022070470120704708B50023406AC385C38401F067FD08BD704790F823
:20598000423007B5222B42D181680268B1F5805F836A3FD1016900293FD15268C2F3080288
:2059A00023F8022B8362C38D013B9BB2C385002B2DD10268D16821F02001D160D16821F41C
:2059C0008071D160516921F001015161202280F842204363026B012A026828D1036302F110
:2059E0000C0353E8003F23F0100302F10C0C4CE800310029F3D11368DB0605D50191136858
:205A0000019353680193019B818DFFF7B7FF03B05DF804FB39B9016929B95268D2B21A7040
:205A2000836A0133BEE7526802F07F02F7E701F005FDECE7036873B51A6804461607D96812
:205A40005D6908D1960668D58D0666D502B0BDE87040FFF794BF05F0010001F49075054378
:205A60005BD0D60705D5CD0542BF636C43F001036364530704D518B1636C43F002036364DA
:205A8000960704D518B1636C43F004036364150707D501F0200303431EBF636C43F00803BB
:205AA0006364636C002B32D0920604D58B0602D52046FFF764FF266820467369626C03F0FA
:205AC000400302F0080253EA020522D0FFF7EAFD73695E0618D5226802F1140353E8003F39
:205AE00023F04003143242E800310029F3D1E06B50B1744B4363FDF757FC40B1E06B436BE0
:205B000002B0BDE870401847204601F09DFC02B070BD01F099FC6564F9E7206B012840F03D
:205B20009480D50640F19180C80640F18E80002201921A6801925A680192019A5A69520652
:205B40004DD5E16B0A68526892B2002ADFD0A08D9042DCD9E2858A69202A36D003F10C022E
:205B600052E8002F22F4807203F10C0040E800210029F3D103F1140252E8002F22F00102F6
:205B800003F1140040E800210029F3D103F1140252E8002F22F0400203F1140040E80021AF
:205BA0000029F3D1202284F84220216303F10C0252E8002F22F0100203F10C0040E800217C
:205BC0000029F3D1E06BFDF7CFFB02236363E38DA18DC91A89B22046FFF7D0FE97E7E28D11
:205BE000E18D92B289B2002991D0A18D891A89B200298CD003F10C0252E8002F22F490721A
:205C000003F10C0545E800200028F3D103F1140252E8002F22F0010203F1140545E8002064
:205C20000028F3D1202284F84220206303F10C0252E8002F22F0100203F10C0545E80020F4
:205C40000028F3D102236363C5E7160628D50D0626D594F84120212A7FF459AFA168226A52
:205C6000B1F5805F17D12169A9B932F8021BC1F3080159602262E28C013A92B2E284002A0D
:205C80007FF445AFDA6822F08002DA60DA6842F04002DA603BE7511C216212785A60EAE776
:205CA00050067FF534AF4A067FF531AFDA68204622F04002DA60202384F8413001F0C1FB80
:205CC00025E700BF6D59000890F84030012B11D02423026880F84130D36823F00C0343F0FC
:205CE0000803D360202380F84130002380F84030184670470220704790F84030012B11D03C
:205D00002423026880F84130D36823F00C0343F00403D360202380F84130002380F84030E8
:205D2000184670470220704790F8412090F84200104370470023C2854364222382850269F0
:205D400080F84230816203681AB1DA6842F48072DA605A69002042F001025A61DA6842F055
:205D60002002DA60704770B590F84260202E07D141B13AB100240463FFF7DCFF204670BDCF
:205D80000220FCE70120FAE7836810B504462BB10322014698470023C4E9023310BD4B1EA0
:205DA000032B00D9FEE78900081F70470139435C13F0100004D0022916D80C4A32F8110026
:205DC000DB0712D503290FD8DFE801F00205080B40F00100704740F01000704740F4807012
:205DE000704740F480507047FEE770472A9700080139032900D9FEE7014B585C704700BF32
:205E0000269700080139032900D9FEE7014B585C704700BF229700082DE9F0410E4604467D
:205E2000FFF7BDFF06F1060805463146204604EB0818FFF7DDFFD8F808302BB1C24323692D
:205E40001A61DA680243DA60771E04EB47039B880B2B49D8DFE803F051181818060618182F
:205E60004A4A4A2AE35DDE0604D5294604F11000FFF714FCE35DD80736D5294604F1100005
:205E8000BDE8F041FFF752BBE35DD90604D5294604F11000FFF7B8FBE35DDA0724D529468B
:205EA00004F11000BDE8F041FFF7F2BA294604F11000FFF73DFB31462046FFF7A3FF014607
:205EC00006462046FFF772FF25692B6A1843D8F80830286243B131462046FFF789FFC34344
:205EE0002B61EB681843E860BDE8F081294604F11000BDE8F041FFF71BBB23691B68DB0703
:205F0000F2D404F11000BDE8F041FFF729B870B5012504462946861C36F8023F23B12946B1
:205F20002046FFF779FF00210135052DF4D1A36E3BB16FF0010223691A61DA6842F0010262
:205F4000DA6049B123691B68DB0705D404F11000BDE87040FFF704B870BD00002DE9F043C1
:205F60008DB0044698460F46FFF719FF4FF6FF731646059305462369C0B95B6B00220693DD
:205F80000123CDE902329DF85030CDE90922079208920B92019204930B2E1DD8DFE806F018
:205FA0000F1545484A5355575B596264042801D19B6BE3E708280CBFDB6B1B6CDEE705927B
:205FC0002A4605A904F1100004E010232A46059305A9E018FFF71CF9013F04EB47039E8037
:205FE00006B3B8F1FF3F1DD0404601F00DF8A84264D140463249083E00F0A0FE032E05D896
:20600000404601F017FF002101F0DAFF40462C4900F0CEFE10F4801F0CBF01221022E35D4E
:206020001343E3550DB0BDE8F08320230593C7E73023FBE760232A4605A904F11000059301
:20604000FFF70CF9C8E77023F5E75023EEE74023ECE7022301932A4601A904F11000FFF7DB
:206060007DF9B9E70A23F5E74046154900F0A0FE10F4801000D0FEE7012304F110092A46A4
:20608000019001A948460293FFF768F939462046FFF7B8FE431EE25C014642F00102E25469
:2060A0000B2204EB43039A8002232046CDE90133FFF775FE01A902464846D0E7FEE700BFAB
:2060C00090980008013903299ABF00EB410080880020704701211030FEF768BF036918685C
:2060E00000F00100704710B502460C46FFF7F6FF80B9CB68DB070ED5CB68104623F00103DD
:20610000CB60FFF7E7FF6FF001032361E36843F00103E36010BD1046BDE81040FFF7DABF25
:206120000B4B98420BD0B0F1804F0AD0A3F59433984208D003F58063984206D0FEE7002069
:20614000704701207047022070470320704700BF002C0140024670B5044652F8100FFFF7BB
:20616000DFFF0546104600F09FFE0023084A04F1600642F82530E36004F1B005B54204D0FC
:20618000103D2846FAF787F8F8E7204670BD00BF98050020F8B504460846FFF7C1FF23695F
:2061A00003B1FEE71B4D04F10C0245F820200E2204F110063046C4E90C33C4E90E33C4E926
:2061C0001033C4E91623216184F82C30A36484F84C3084F84D30E46000F022FE04F1600596
:2061E00004F1B00728461035FFF7CEFDBD42F9D100234FF6FF72C4E90033C4E90632C4E96B
:206200000833A360636180233046A362BDE8F840FEF7A6BF9805002010B586B014220446EF
:20622000002101A802F034F90023694601A80093FEF704FE206900F0CDFE012802D0022807
:206240000FD0FEE7049CFEF7D9FDB4F5C06F05D00BD824F48074B4F5806F00D1400006B014
:2062600010BD059CFEF7DAFDEFE7B4F5E06FF4E7012A38B505460C460BD0022A16D004B1E4
:20628000013C29692846CC62EC61BDE83840FFF72ABFFFF7C1FF084BB0FBF3F044432A6999
:2062A000230C93620133B4FBF3F4E8E7FFF7B4FFB0FBF4F4F3E700BF40420F00F8B50546C3
:2062C00014461A46FFF76BFD2B69822A9E6A074606F1010629D01FD8102A11D852BB4FF6AE
:2062E000FF722969CB6A934203D1B4F5803F08BF1C4637BB4C632846BDE8F840FFF7F3BE99
:20630000812AECD12846FFF787FF124BB0FBF3F06043B0FBF6F4E2E7832AE0D1DB6A03FB9E
:2063200004436424B3FBF4F4D9E72846FFF774FF6643EEE7DB6A03FB044301249440013C23
:20634000F0E7042F01D18C63D5E7082F0CBFCC630C64D0E740420F00034B186810B104300A
:20636000FEF738BE704700BF98050020FFF7F4BF034B586810B10430FEF72CBE704700BFFE
:2063800098050020034B986810B10430FEF722BE704700BF98050020034BD86810B1043072
:2063A000FEF718BE704700BF980500200022C0E90022C0E902227047F8B504460E4600F132
:2063C000600500F1B00728461035FFF7EFFFBD42F9D10023204631462361FFF7DBFE204697
:2063E000F8BD826810B50AB902F048FCC368BDE81040184708B500B9FEE700F00FFD006802
:20640000836E13B16030FFF7ECFF08BDFFF7F2BF10B500B9FEE7037F013B072B10D8DFE8E8
:2064200003F004140F100F0F0F12012400F0F6FC0068063400EB041083680BB1FFF7D1FFDE
:2064400010BD0324F2E70424F0E70224EEE7FFF7DFBFFFF7DDBF01F0ABBE01F0B1BE000095
:2064600086B0042841D8DFE800F003101C2834001F4B20489A6942F004029A619B6903F060
:2064800004030193019B06B07047194B1A489A6942F008029A619B6903F008030293029B24
:2064A000F1E7134B15489A6942F010029A619B6903F010030393039BE5E70D4B10489A694A
:2064C00042F020029A619B6903F020030493049BD9E7074B0B489A6942F040029A619B6942
:2064E00003F040030593059BCDE70020CBE700BF0010024000080140000C014000100140B0
:2065000000140140001801402DE9F3478A46244999469046064600F029FCFFF701FE214FC5
:20652000054657F8203073B9B020FFF794FF1C490446304600F01AFC01462046FFF73CFFE3
:2065400057F825301C60164930461C6800F030FCC0F3C43529462046FFF7B4FD0428074605
:2065600007D0002304220093294633462046FFF7F5FC022251462046FFF77AFE4B4642468B
:2065800029462046FFF79AFE042F05D0204602B0BDE8F047FFF7BBBC02B0BDE8F08700BFA2
:2065A0009098000898050020F8B51349064600F0DDFBFFF7B5FD114F054657F8203073B9B3
:2065C000B020FFF748FF0C490446304600F0CEFB01462046FFF7F0FE57F825301C601C68AB
:2065E00044B12046FFF7B6FD2046BDE8F840B021FFF733BFF8BD00BF90980008980500203A
:20660000FCF712BE704708B5FCF702FEFCF797FEFFF7F8FF08BD70470F4B84B0DA6942F05C
:206620008052DA61DA6902F080520192019A9A6942F001029A619A6902F001020292029ABD
:206640005A6942F040025A615B6903F040030393039B04B0704700BF001002400C4BD3F87C
:20666000FC20D2015EBFD3F8FC2042F08072C3F8FC200022074B5A601A6842F001021A60CD
:2066800000BF00BF00BF5868B0FA80F04009704700ED00E0001000E008B5FFF7BDFFFFF7C1
:2066A000DDFFFCF7A3FDFFF7B6FF00F05DFFBDE808400148FCF748BE200000200023C0E939
:2066C0000033C0E9023370472DE9F043164600270A468BB0012A07F101046ED1CDE9021369
:2066E0000023FF2998BF02461D461C464FF0010C88BF021D0CFA03FE714505D11D46FF291B
:206700004FEA830488BF203C0133102BF2D10F231268A34013400822A240934250D10123DC
:20672000C268AB4093430CBF0123022304930323142402A90593FCF781FE0023FFB27C431D
:20674000DFF88480D6F80890043406AD06934444C5E901330993B9F1000F33D00222314617
:206760002846C847D6E9029C95E8030014267E43CDE9000108EB0603043393E8030085E8EF
:206780000300DDE9000183E80300A36828460893E368C4F80890C4F80CC00993F9F77BFD82
:2067A0000022062118F90600FCF756FD18F90600FCF782FD0BB0BDE8F0832746520889E7A0
:2067C0000023B3E7CC46CFE7A80500200023012803F101020AD11422DBB25343054A181D6C
:2067E0001044816829B11A441369184713464008EDE77047A80500200120FCF7F3BE022069
:20680000FCF7F0BE0420FCF7EDBE0820FCF7EABE1020FCF7E7BE08B52020FCF7E3FE402059
:20682000FCF7E0FE8020FCF7DDFE4FF48070FCF7D9FEBDE808404FF40070FCF7D3BE38B50B
:2068400006244FF48065A8B2FCF7CCFE013C4FEA4505F8D138BD0000344A08B51046062397
:2068600000F8043BFFF72AFF072302F118001375FFF724FF082302F12C0082F82830FFF7DA
:206880001DFF092302F1400082F83C30FFF716FF0A23172102F1540082F85030FFF70EFFE3
:2068A00002F1680082F86410FFF708FF02F17C0082F87810FFF702FF02F1900082F88C1091
:2068C000FFF7FCFE02F1A40082F8A010FFF7F6FE82F8B410282102F1B800FFF7EFFE02F115
:2068E000CC0082F8C810FFF7E9FE02F1E00082F8DC10FFF7E3FE02F1F40082F8F010FFF736
:20690000DDFE02F5847082F80411FFF7D7FE02F58E7082F81811FFF7D1FEBDE8084002F516
:20692000987082F82C11FFF7C9BE00BFA805002038B5054CA4F5A075143C201DF9F7ABFC7F
:20694000AC42F9D138BD00BFE80600207B4B82B09A69013842F001029A619B6903F001035E
:206960000193019B23282CD8DFE810F024002D0034003B00400047004C00530058005F0034
:2069800068006D0074007D008200890092009B00A000A700B000B500BC002B002B002B0010
:2069A000C100C8002B002B002B002B00CD00D200D900E000624A536843F0E06343F0010336
:2069C000536002B070475E4A536823F0010343F0E063F5E75A4A536843F0E06343F00203C2
:2069E000EEE7574A536823F00203F0E7544A536843F0E06343F00403E2E7514A536823F03C
:206A00000403E4E74E4A536843F0E06343F00803D6E74B4A536823F00803D8E7484A536866
:206A200043F0E06343F03003CAE7454A536823F0300343F0E06343F01003C1E7404A536890
:206A400023F03003C3E73E4A536843F0E06343F0C003B5E73A4A536823F0C00343F0E06370
:206A600043F04003ACE7364A536823F0C003AEE7334A536843F0E06343F44073A0E7304ACE
:206A8000536823F4407343F0E06343F4007397E72B4A536823F4407343F0E06343F4807339
:206AA0008EE7274A536823F4407390E7244A536843F0E06343F4406382E7214A536823F4D5
:206AC000406343F0E06343F4006379E71C4A536823F440637BE71A4A536843F0E06343F49A
:206AE00080536DE7164A536823F480536FE7144A536843F0E06343F4004361E7104A5368AE
:206B000023F4004363E70E4A536823F0E06357E70B4A536823F0E06343F0807350E7084A15
:206B2000536823F0E06343F0007349E7044A536823F0E06343F0806342E700BF00100240BF
:206B40000000014091FAA1F3B3FA83F370B50D0E0F2691FAA1F1B1FA81F144599B0006FACB
:206B600003F3890024EA03048A402243425170BD91FAA1F3B3FA83F370B50D0E042691FA5B
:206B8000A1F1B1FA81F144599B0006FA03F3890024EA03048A402243425170BD431C04D058
:206BA0000C3151F80C3C5A1C01D100207047834201F10C01F5D1012070470000431C2DE911
:206BC000F34106460F4600D1FEE7594B00F00F02C0F3031001F0070853F82240FFF740FCE0
:206BE000B8F1010F054615D194FAA4F3B3FA83F30321200E2A589B0001FA03F322EA0302F2
:206C000094FAA4F3B3FA83F39B00994011432950012213E0C7F30620B8F1030F0AD801A3B4
:206C200053F828F0376C0008116C00089B6C0008A96C0008FEE7FFF789FE08222146284634
:206C400008F1FF38FFF77EFFB8F1010F06D817F0080218BF04222146FFF78AFF94FAA4F2E2
:206C6000230EB2FA82F2E9580F239200934094FAA4F2B2FA82F2C7F301170B409200012FC8
:206C800023FA02F312D0022F3BD0082B21D1042221462846FFF756FF1BE07F2801D10922BA
:206CA000CCE7FFF753FEFAE70022C7E7042B04D1082221462846FFF745FF230A93FAA3F39C
:206CC000B3FA83F20123E968934021EA14210B43EB60184B9A6942F001029A619B6903F0E4
:206CE00001030193019BA6F10D03012B14D8124A536823F0E06343F08063536002B0BDE814
:206D0000F081042B04D1082221462846FFF71AFFEB6823EA1423DBE70F2E02D0133E012E08
:206D2000ECD8054A536823F0E06343F00073E4E7309700080010024000000140431C06D126
:206D40007047834202D18968FFF738BF0C310B685A1CF6D1FEE70B685A1C01D100207047A2
:206D6000834201D1486870470C31F4E7431C01D0FFF7F1BF002070474B6813B94FF0FF3063
:206D80007047834201D1086870470C31F4E708B1FFF7F2BF4FF0FF30704703460868421CCA
:206DA00000D17047984201D1886870470C31F5E7431C01D0FFF7F1BF704703468B420846EE
:206DC00004D01BB100290CBF18460020704700000F4B1A6842F001021A6059680D4A0A40FD
:206DE0005A601A6822F0847222F480321A601A6822F480221A605A6822F4FE025A604FF484
:206E00001F029A604FF00062034B9A60704700BF001002400000FFF800ED00E004387047EF
:206E200003681D4A84B093420BD11C4B9A6942F400629A619B6903F400630093009B04B05E
:206E40007047B3F1804F0BD103F50433DA6942F00102DA61DB6903F001030193019BEEE70A
:206E60000F4A93420AD10D4BDA6942F00202DA61DB6903F002030293029BE0E7094A9342A0
:206E8000DDD1064BDA6942F00402DA61DB6903F004030393039BD2E7002C01400010024053
:206EA00000040040000800400368124A934206D102F56442936923F4006393617047B3F171
:206EC000804F05D10C4AD36923F00103D36170470A4A934205D102F50332D36923F00203FA
:206EE000F4E7074A9342F2D102F50232D36923F00403EBE7002C0140001002400004004078
:206F000000080040431C10D00C4B984210D007D8B0F1804F0ED0A3F5806398420CD0FEE796
:206F2000074B9842FBD1192070476FF00D0070471E2070471C2070471D2070470008004022
:206F4000002C0140431C10D00C4B984210D007D8B0F1804F0ED0A3F5806398420CD0FEE731
:206F6000074B9842FBD11B2070476FF00D0070471E2070471C2070471D20704700080040E0
:206F8000002C014038B50446FFF74AFF0068FFF7B9FFD4E91212FCF75FF92068FFF7B2FF9D
:206FA000FCF78AF922681046FFF7CCFF05461046FFF7A8FF85420BD0D4E912122846FCF798
:206FC0004BF92068FFF7BEFFBDE83840FCF774B938BD0000431C0CD0094B98420BD007D8DD
:206FE00020F48063B3F1804F07D0064B984204D0FEE700207047022070470120704700BF25
:20700000002C01400008004008B50649FFF7D0FEC0F3C430431E032B00D9FEE7800004383B
:2070200008BD00BF909800082DE9F04F87B09846109B04468A46406D664991460193FFF7B0
:2070400095FE65498346A06DFFF790FE63490646E06DFFF78BFE62490546206EFFF786FED3
:207060000746BBF1000F00F0B180A26D013202D0002E00F0AB80E26D013202D0002D00F019
:20708000A580226E013202D0002F00F09F8031465846FFF792FE0346206020B90146FFF77E
:2070A0008CFE0346206029461846FFF786FE39462060FFF782FE2060002800F08780494B8E
:2070C00098424CD103F55843DA6842F48042DA60DA6822F48042DA609A6942F480429A6168
:2070E0009B6903F480430393039B2523A4F864303849606DFFF722FE1EB13749A06DFFF770
:207100001DFE2DB13549E06DFFF718FE4FF480752FB13349206E45F40075FFF70FFE94F840
:207120006520314B271D43F8227023680022C4E9013A019B94F96400C4E904380C230121E1
:20714000C4E90635C4F80C902262FCF785F83846002E36D107B0BDE8F04FFEF76DBB234B22
:20716000984215D103F5E6331A6942F400321A611A6922F400321A61DA6942F40032DA61AC
:20718000DB6903F400330493049B4FF49373ADE7174B9842ACD103F5E4331A6942F480224B
:2071A0001A611A6922F480221A61DA6942F48022DA61DB6903F480230593059B40F22723B6
:2071C00094E707B0BDE8F04FFEF707BB07B0BDE8F08F00BF4898000800980008C49700085D
:2071E0008897000800380140E8060020004400400048004010B4019C18B1019410BCFFF754
:2072000013BF10BC704700000A4A0B4B926813B553F8224009492046FFF7A8FD40B1002399
:2072200007481A4644654FF416510093FFF7FCFE02B010BD249B0008649B00084898000894
:207240002C00002008B5074B90F8652053F82200FEF76AFD00F02200A0F122035842584102
:2072600008BD00BFE806002008B5074B90F8652053F82200FEF758FD00F02100A0F12103E3
:207280005842584108BD00BFE80600202DE9F84306460C46FBF7C8FF274D074695F865309E
:2072A000022B2ED9254A264B9268264953F822804046FFF75BFDF0B900242046BDE8F8833D
:2072C00059F8232052B140461E49FFF74FFD95F8653059F823201268824210D00133DBB253
:2072E000022B85F86530EBD9FFF78EFF95F86530022B06D9E0E70023DFF84C90F0E7022B39
:20730000F2D8114A52F82350A5F104084046FFF7ABFF48B94FF47A7331462846A2B2FEF764
:20732000BEFA0028C8D1C8E7FBF77EFFC01BB0F57A7FEBD3C0E700BF2C000020249B000806
:20734000649B000848980008E806002070B50E46054610B94FF0FF3070BDFFF773FF044656
:207360000028F7D1294611F8663F0122337095F86500034B53F82000FEF7F5FC2046EBE771
:20738000E806002038B50D460446B8B1FFF75AFFA0B994F96400E564FBF79CFF94F865008C
:2073A000074B04F1660153F820000122FEF7DBFC94F96400BDE83840FBF77EBF38BD00BFD4
:2073C000E806002038B515460446B8B1016590F96400FBF77FFFB4F87630E16E9BB294F867
:2073E00065001944064BAAB253F82000FEF7A5FA94F96400BDE83840FBF75EBF38BD00BF4E
:20740000E806002048B1836D013306D190F86520024B53F82200FEF757BC7047E8060020D6
:2074200048B1836D013306D190F86520024B53F82200FEF761BC7047E8060020836C04388F
:207440001847C36C0438184730B5044650F8043985B01D6815F0010512D0002200921A6872
:2074600000925B680093009BFFF7ECFE40BB0122204604F1620105B0BDE83040FEF773BCDF
:20748000196811F0020106D001951A6801925B680193019BE8E71A6812F0040206D0029131
:2074A0001A6802925B680293029BDDE719680907DAD503921A6803925B680393039BD3E760
:2074C00005B030BD08B52520FBF72AFF024B1868BDE80840FEF7AEBAE8060020262008B5C5
:2074E000FBF71EFF034B586818B1BDE80840FEF7A1BA08BDE8060020272008B5FBF710FF91
:20750000034B986818B1BDE80840FEF793BA08BDE806002003460A4910B508680344EFF358
:207520000882934205D90C224FF0FF30054B1A6010BD054A054C121B9342F4D20B60F7E72A
:20754000A8000020600900200050002000040000FEE700001622024B4FF0FF301A6070475D
:20756000600900200120704710B590B02022002107A800F08DFF1422002101A800F088FFA0
:20758000102301220224CDE90A234FF4601306A806940D940F93FDF7D3F900B1FEE70F23C3
:2075A000CDE901344FF480630390CDE90430214601A8FDF787FB00B1FEE710B010BDB0F8EC
:2075C0000831B0F80421981A00F03F007047B0F80831B0F804219BB293421ABFD0F8FC3070
:2075E000985C4FF0FF30704790F80631B0F80A01C0B2834227BFC3F13F03C018C01A00F14A
:20760000FF30704707B503688DF8071001225B680DF10701984703B05DF804FB13B50DF129
:2076200007010446FFF792FE88B9B4F87430B4F87020013303F03F03934208D0B4F874204F
:207640009DF80700A16E92B28854A4F8743002B010BD0000B0F87610826F10B50A4402F07C
:207660003F02A0F87620B0F87610B0F8722089B28A421AD0B0F876404032A4B2B0F87610EE
:20768000121B544289B204F03F0402F03F02C1F1400158BF62428A4228BF0A46044982679B
:2076A000FFF790FE4FF0FF3010BD0020FCE700BF557600082DE9F843036804469B6888469F
:2076C0001646984701232374D4F8EC30B4F8067101338146C7F1400709D194F8103133B124
:2076E000002304F1940084F81031FFF78BFE236820469B6898470028F9D03546BD4225D867
:207700004D4523D8B4F80631D4F800015A19402A184430D82A46414600F00AFF2F46B4F8DA
:2077200006311D4405F03F05A4F8065104F194052846FFF799FD30B93A4628461549C4F80C
:207740000C71FFF73FFE3046BDE8F8834F4528BF4F4623683A4641465B68204698472368AE
:2077600020469B689847ED1BB844B4F806718146C7F14007C2E7C3F140073A46414600F039
:20778000D7FED4F80001EA1B08EB070100F0D0FEC5E700BF55760008C0F8F030009B914205
:2077A00008BF4FF0FF31C0F8F43000F11103C0F8FC300023C0E93A2100F15102A0F8083192
:2077C000C0E94023A0F80A317047000073B54FF47A750026C0E901653D4D069C0560CDB274
:2077E000322D25D83B4E01F4E06156F825502943D5B2322D30D8374E02F4E06256F82550D1
:207800002A43DDB2322D3BD8324E03F4E06356F825502B43E5B2322D46D82E4E04F4E06443
:2078200056F825502C430094FFF7B6FF02B070BD01F0C006C02E0CD1CF2D0AD8264D01F034
:207840003F0655F82660234D01F4E06155F82650CDE74FF0FF31CBE702F0C006C02E0CD14F
:20786000CF2D0AD81C4D02F03F0655F82660194D02F4E06255F82650C2E74FF0FF32C0E796
:2078800003F0C006C02E0CD1CF2D0AD8124D03F03F0655F826600F4D03F4E06355F82650C3
:2078A000B7E74FF0FF33B5E704F0C006C02E0CD1CF2D0AD8084D04F03F0655F82660054D07
:2078C00004F4E06455F82650ACE74FF0FF34AAE7409C0008649B0008249B0008037C70B5BD
:2078E00004460D46A3B1FBF79FFC0646B4F80621B4F80A319BB29A420AD0002DF8D0FBF71A
:2079000093FC801B8542F1D8B4F80A31A4F8063170BD0021FFF7E2BFCBB2322B08D80E4AFC
:2079200001F4E06152F823301943C0F8EC10704701F0C002C02A0CD1CF2B0AD8074B01F014
:207940003F0253F82220044B01F4E06153F82230EAE74FF0FF31E8E7649B0008249B00085A
:20796000CBB2322B08D80E4A01F4E06152F823301943C0F8E810704701F0C002C02A0CD1E5
:20798000CF2B0AD8074B01F03F0253F82220044B01F4E06153F82230EAE74FF0FF31E8E7C9
:2079A000649B0008249B000873B54FF47A7316460022C0E901231D4B044603604FF0FF33D0
:2079C000C0F8EC301A4B0D46984215D1C321FFF7A3FFC221FFF7C4FF4FF0FF33012E08BFDC
:2079E000C4F8EC3000932046D4E93A214FF0FF33FFF7D2FE02B070BD0E4B0F499A680F4B7B
:207A000053F82200FFF7B2F9854202D1C3212046DDE70B492846FFF7BAF90749C4F8EC004D
:207A20002846FFF7B4F9C4F8E800D5E7409C0008F4060020249B000848980008649B000821
:207A400000980008D0F8EC3010B5013304460ED10368DB68984794F8103143B9012304F111
:207A6000940084F81031BDE81040FFF7D9BC10BD73B5144602F00703023BDBB2042B80F879
:207A8000112196BF1A4A0022D25C04F03003302B0546C0F8141107D14FF4C0630132082A5E
:207AA00009D0092A1BD0FEE714F020031CD04FF480630132F3E70022C4F3C00405F1940677
:207AC000640330460094FFF795FB2846FFF7BAFF3046084902B0BDE87040FFF753BC4FF47C
:207AE0008052E9E71A46E7E7082AFBD0DBE700BF309C00081D76000810B50446FFF7A2FF23
:207B0000B4F80821B4F8043192B29A4217BFD4F8FC204FF0FF30D05C01331CBF03F03F03F3
:207B2000A4F8043110BD0000002202490248FFF73BBF00BF00440040F406002070B5054633
:207B40000C46084649B1F8F7E1FA2B68024621462846BDE870405B68184770BD08B5FFF7BA
:207B6000EDFF08BD03681B681847000008B50249FFF7E4FF08BD00BFC394000838B505460B
:207B8000FFF7DCFF04462846FFF7F0FF204438BDFFF7F4BF70B50D46144630B1461E012E2F
:207BA00005D811462846FFF771FB204670BD03685B689847F9E70EB403B503AA52F8041BB1
:207BC000019200F013FC02B05DF804EB03B070470023012A98BF0A2230B58BB00C468DF8EB
:207BE000243009A92546B4FBF2F404FB1253DBB2092B94BF30333733DBB2AA4201F8013D8A
:207C0000F0D9FFF79BFF0BB030BD2DE9F04107460E4614462AB9BDE8F0410368C9B21B68FF
:207C200018470A2A05D1002905DBBDE8F041FFF7CFBFD2B2F9E72D21FFF794FF224605468A
:207C400071423846FFF7C4FF2844BDE8F081FFF7DCBF10B422B9026810BC1268C9B2104706
:207C600010BCD2B2FFF7B4BFFFF7F3BF38B50546FFF7EFFF04462846FFF778FF204438BD09
:207C800010B5044600F072FAE060236820465B699847002808DA00F069FAE368C01AA36818
:207CA0009842F2D34FF0FF3010BDF8B507460D460C468E18B44201D1601BF8BD3846FFF739
:207CC000DFFF431CF8D004F8010BF3E72DE9F0410746884616461D4673B100243846FFF7E0
:207CE000CFFF431C05D0404503D030550134A542F4D12046BDE8F0811C46FAE72DE9F041BE
:207D0000C3B2322B0D46904686B04ED8394A00F4E06452F823301C43C4F30310FEF7A0FBFB
:207D2000074600283ED0B8F1020F52D0B8F1030F51D0314E314BB8F1000F08BF1E46304BAF
:207D40009A6942F001029A619B6903F001030193019BA4F10D03012B3FD82A4A536823F09B
:207D6000E06343F08063536000230122CDE90233CDE9043304F00F04AB6802FA04F4A4B275
:207D80003BB10222294602A89847EB680593AB68049338463346214602AAFEF795FC02A80C
:207DA000F8F779FA06B0BDE8F08100F0C002C02A0CD1CF2B0AD8144B00F03F0253F8222023
:207DC0000C4B00F4E06453F82230A4E74FF0FF34A2E70E4EB3E7094EB1E70F2C03D0A4F169
:207DE0001303012BC0D8074A536823F0E06343F00073B8E7649B00080000111000002110A9
:207E00000010024000000140249B00080000311008B50320FBF70EFABDE8084000F0C4B993
:207E200008B5AFF30080F9F7E1FEFAF7CBFB00F0ADF9FAE7C0F30312042A034610B50ED87C
:207E40000020084AD9B252F8044B8C4203D103F4E063184310BD01303328F4D1FAE7332003
:207E6000F8E700BF649B0008FEF7B2FF0B480C490C4A002302E0D458C4500433C4188C4293
:207E8000F9D3094A094C002301E013600432A242FBD300F027FBFFF7C3FF7047000000206E
:207EA00008010020949C00080801002068090020FEE791420FD008D90123891A8B409842C3
:207EC00008D30130C8400138704720B10130521A9040F8E700207047014B1860704700BF70
:207EE000AC000020C3B2322B2DE9F04107460E4631D82C4A00F4E06452F823301C43621CCB
:207F00004ED020462849FEF749FEDFF8A0800546002831D0264AC4F3031152F8210004F02B
:207F20000F0520FA05F3DB075FBF0123AB40034342F821301F4BD8F800101D6830462A4686
:207F4000FFF7B7FF1C490246EBB22046BDE8F0410968FEF7D9BA00F0C002C02A20D1CF2B6F
:207F60001ED8164B00F03F0253F822200D4B00F4E06453F82230C1E73846012100F020F86F
:207F8000D8F8001030460822FFF793FF7F2898BF29463846BDE8F04188BF012100F06EB899
:207FA000BDE8F081649B000890980008B40000200C080020B0000020AC000020249B000809
:207FC000C3B2322B2DE9F0410D462AD8274A00F4E06452F823301C43621C44D0244EC4F3D3
:207FE000031756F8273004F00F0823FA08F3DB0710D520461F49FEF7D1FD10B12046FEF72B
:20800000D3FA012256F8273002FA08F223EA020346F82730052D15D8DFE805F015211B1DE5
:208020001F2300F0C002C02A1DD1CF2B1BD8124B00F03F0253F822200C4B00F4E06453F892
:208040002230C8E7FEE700212046BDE8F041FEF7B5BD1021F8E72021F6E70321F4E7012127
:20806000F2E70921F0E7BDE8F08100BF649B00080C08002090980008249B0008C3B2322B4D
:208080001BD8174A00F4E06052F823301843431C25D0C0F30313042B98BF124A00F00F0062
:2080A00098BF52F82320104B88BF002253F82030C3F30F2391B11361704700F0C002C02A8C
:2080C0000DD1CF2B0BD8094B00F03F0253F82220034B00F4E06053F82230D7E7536170478B
:2080E000649B00080C00002030970008249B0008C3B2322B1CD8194A00F4E06052F82330BD
:208100001843431C25D0C0F30313042B23D8144A00F00F0052F82330124A9B6852F82020DA
:20812000D84300EA122080B2B0FA80F04009704700F0C002C02A0CD1CF2B0AD80A4B00F022
:208140003F0253F82220054B00F4E06053F82230D6E70020704700239B68FFDE649B000892
:208160000C00002030970008249B0008FEF748BA38B5044648B1FEF743FA054600F016F89B
:20818000FEF73EFA431BA342F8D338BD08B5044B2BB10448FFF713FA08B1AFF3008008BDD8
:2081A00000000000F4060020FEF776BA70470000024B0146186800F02DB800BFB800002049
:2081C000024B0146186800F0C1B900BFB800002070B50F4E0C463168054611B900F060F9BF
:2081E00030602146284600F05BF9431C03D14FF0FF34204670BDC41C24F00304A042F8D0F9
:20820000211A284600F04CF90130F2D1EFE700BF200800202DE9F843CD1C25F0030508351B
:208220000C2D38BF0C25002D064601DBA94204D90C2333600020BDE8F883DFF8D48000F0A3
:2082400069F8D8F800301C4644BB29463046FFF7BFFF431C044658D1D8F800402746002F45
:2082600043D1002C4BD023683946304604EB030900F016F9814542D1216830466D1A29465B
:20828000FFF7A6FF01303AD023682B442360D8F800305A6862BBC8F800700FE02268521B96
:2082A00020D40B2A17D96119A342256018BF5960636808BFC8F8001062514B60304600F00B
:2082C0002FF804F10B00231D20F00700C21A1CBF1B1AA350AFE76268A3420CBFC8F8002051
:2082E0005A60EBE723466468AEE73C467F68B6E71A465B68A342FBD100235360DEE70C2384
:208300003046336000F00CF894E70560D6E700BF24080020014800F009B900BF6409002071
:20832000014800F004B900BF64090020024B0A460146186800F002B8B80000202DE9F041CE
:20834000074614460D4621B91146BDE8F041FFF761BF2AB900F0FAF825462846BDE8F08152
:2083600000F03CF98442064602D8B4EB500FF4D821463846FFF74EFF804608B94546ECE715
:20838000B4422246294628BF324600F0D1F82946384600F0DBF8F1E72DE9F0410F464FF491
:2083A0000071ADF5047D03AD0DF1100829600093414613462A46064600F022F8044688B11E
:2083C0000246394630462B6800F07AF84445286003D02146304600F0B9F828680DF5047DF6
:2083E000BDE8F0814FF0FF30F8E7000013460A46014602480068FFF7CFBF00BFB80000205D
:2084000070B515469AB01A4689B12C689CB94FF4227321460026B442ADF80C301996009193
:2084200004910BDA8B23036000201AB070BD4FF422730C46EEE74FF4C163EBE74FF6FF73AB
:208440006946ADF80E301E9B0294059400F02EF90028E9DB009B28601E700498E5E78842BC
:2084600010B501EB020402D98442234607D8431EA14207D011F8012B03F8012FF8E70244BC
:20848000824200D110BD13F8011D02F8011DF7E703460244934200D1704703F8011BF9E778
:2084A00038B50023054D044608462B60FFF732F8431C02D12B6803B1236038BD600900209D
:2084C00038B50446084611460022054D2A601A46FFF760FB431C02D12B6803B1236038BD20
:2084E0006009002070B500260C4D0D4B5B1B9C10A64209D1002600F0C5FB0A4D0A4B5B1B1B
:208500009C10A64205D170BD55F8043B98470136EEE755F8043B98470136F2E76C9C0008C2
:208520006C9C00086C9C0008849C0008704770470A44914200F1FF3300D1704710B511F8EB
:20854000014B914203F8014FF9D110BD38B50546002940D051F8043C0C1F002BB8BFE41857
:20856000FFF7D8FE1C4A136833B9636014602846BDE83840FFF7D4BEA34208D92068211891
:208580008B4201BF19685B6809182160EDE71A465B680BB1A342FAD911685018A0420BD15E
:2085A00020680144501883421160E0D118685B68084410605360DAE702D90C232B60D6E7DA
:2085C000206821188B4201BF19685B680918216063605460CBE738BD2408002051F8043C74
:2085E000181F002BBCBF0B58C01870472DE9F0471F468E688246BE420C469046334653D870
:20860000B1F90C0010F4906F2BD065692368096905EB4505A3EB010905EBD5757B1C6D10BB
:208620004B44AB422A4684BF1D462A46430527D511465046FFF7EEFD064658B34A462169B5
:20864000FFF776FFA38923F4906343F08003A38126614E4426603B463E466561A5EB090597
:20866000A5601F463A4641462068FFF7F8FE0020A3689B1BA36023683B442360BDE8F08788
:208680005046FFF75BFE06460028E1D150462169FFF75CFF0C23CAF80030A3894FF0FF30A3
:2086A00043F04003A381E9E73E46DBE72DE9F04F98468B8907461B060D4614469DB010D576
:2086C0000B6973B94021FFF7A5FD2860286130B90C233B604FF0FF301DB0BDE8F08F40237B
:2086E0006B610023099320238DF8293030234FF00109CDF80C80DFF898818DF82A302346A9
:208700009A4613F8012B0AB1252AF9D1BAEB040B0BD05B46224629463846FFF767FF01305C
:2087200000F0A780099A5A4409929AF80030002B00F09F8000234FF0FF32CDE905230AF1DE
:20874000010A049307938DF853301A935446052214F8011B4E4800F037FA049AD8B9D00683
:2087600044BF20238DF85330110744BF2B238DF853309AF800302A2B15D0544600204FF045
:208780000A0C079A214611F8013B303B092B4BD9B0B1079214E0A0EB080309FA03F31343E0
:2087A000A2460493D2E7039B191D1B680391002BBBBF5B4242F0020207930793B8BF0492DD
:2087C00023782E2B0AD163782A2B32D1039B02341A1D1B68039243EAE3730593DFF8B4A02E
:2087E00003225046217800F0EFF938B14022049BA0EB0A00824013430134049314F8011BC2
:20880000062225488DF8281000F0DEF9002836D0224B1BBB039B073323F007030833039308
:20882000099B334409936AE70C4601200CFB0232A8E700234FF00A0C1946013405932046E9
:2088400010F8012B303A092A03D9002BC6D00591C4E7044601230CFB0121F0E703AB0093BA
:208860002A4638460E4B04A9AFF30080421C0646D6D1AB895B063FF52DAF09982CE703AB8A
:2088800000932A463846064B04A900F07DF8EDE7C6940008CC940008D094000800000000EA
:2088A000ED8500082DE9F047164698468A680B6907469342B8BF1346336091F843200C468E
:2088C000DDF820900AB1013333602368990642BF336802333360256815F0060506D104F19A
:2088E000190AE36832689B1AAB422BDC94F843302268003B18BF0123920630D44146384667
:2089000004F14302C847013023D02368226903F00603042B14BF002533684FF0000608BF0A
:20892000E56804F11A0408BFED1A54F8123C08BF25EAE5759342C4BF9B1AED18B5421AD14B
:20894000002008E00123524641463846C847013003D14FF0FF30BDE8F0870135C1E7302082
:20896000E11881F843005A1C94F845102244023382F84310C2E70123224641463846C8473A
:208980000130E6D00136D9E72DE9FF470F7E9146782F80460C469A460C9E01F1430207D8DA
:2089A000622F0AD8002F00F0D280582F00F0B78004F1420684F842703AE0A7F16303152B62
:2089C000F6D801A151F823F0218A0008358A0008B1890008B1890008B1890008B189000849
:2089E000358A0008B1890008B1890008B1890008B1890008358B00085F8A0008EB8A000872
:208A0000B1890008B1890008578B0008B18900085F8A0008B1890008B1890008F38A0008AC
:208A200033681A1D1B68326004F1420684F8423001239DE033682068191D3160060601D5B7
:208A40001D6803E04506FBD5B3F90050002D03DA2D236D4284F843300A23594810E0216858
:208A60003368080653F8045B02D4490648BFADB26F2F5348336059D10823002184F8431007
:208A80006668002EA66005DB21682E4321F0040121604DD01646B5FBF3F103FB1157C75DCC
:208AA00006F8017D2F46BB420D46F4D9082B0BD12368DF0708D5236961689942DEBF30232B
:208AC00006F8013C06F1FF36921B22614B4621464046CDF800A003AAFFF7E4FE01304CD149
:208AE0004FF0FF3004B0BDE8F087236843F0200323607827334884F84570236831681F0640
:208B000051F8045B02D45F0648BFADB23160D90744BF43F0200323601DB11023ADE72848BA
:208B2000E9E7236823F020032360F6E70A23A4E71646BBE733682568181D616930602E06A3
:208B40001B6801D5196002E06806FBD51980002316462361BAE7336800211A1D32601E68DB
:208B60006268304600F030F808B1801B606063682361002384F84330A8E73246494640460C
:208B80002369D0470130ABD023689B0713D4E068039B9842B8BF1846A4E701233246494627
:208BA0004046D04701309BD00135E36803995B1AAB42F2DCEBE7002504F11906F5E700BF89
:208BC000D7940008E8940008034610B5C9B202449342184601D1002003E0047801338C4249
:208BE000F6D110BD062008B500F02CF80120FEF7AFFC1F2938B505460C4604D916230360DE
:208C00004FF0FF3038BDC26B12B152F821304BB9284600F031F8224601462846BDE83840A1
:208C200000F018B8012B0AD0591C03D1162303600120E7E70021204642F8241098470020A6
:208C4000E0E70000024B01461868FFF7D2BF00BFB800002038B50023064D044608461146C9
:208C60002B60FEF777FC431C02D12B6803B1236038BD00BF60090020FEF774BC08B5FFF7F0
:208C8000B1FF0000F8B500BFF8BC08BC9E467047F8B500BFF8BC08BC9E4670477E58506F91
:208CA0007765727341585032313031005344413A25642053434C3A256400486561645068BC
:208CC0006F6E65206465746563746564004D697374616B6520212054686520737465707351
:208CE000206973206D757374202575206D56004D697374616B65202120546865206D696E3E
:208D0000696D756D207365747461626C6520766F6C74616765206F662056535953206973AF
:208D2000202575206D56004D697374616B65202120546865206D6178696D756D20736574BC
:208D40007461626C6520766F6C74616765206F662056535953206973202575206D560046B0
:208D600061696C656420746F2064697361626C652074686520706F776572206368616E6E27
:208D8000656C2C2074686520706F776572206368616E6E656C20686173206265656E207089
:208DA000726F74656374656400454E41424C450044495341424C45002573202D20484558D4
:208DC0003A30782578200A004D697374616B6520212020546865207374657073206973200F
:208DE0006D7573742025756D56004D697374616B6520212054686520737465707320697392
:208E0000206D7573742025756D56004D697374616B65202120444335206D696E696D756DE5
:208E200020766F6C746167652069732025756D56202C25756D56004D697374616B652021EF
:208E400020444335206D6178696D756D20766F6C746167652069732025756D56004D697364
:208E600074616B65202120424C444F31206D696E696D756D206F757470757420766F6C74C8
:208E8000616765206973202025756D56004D697374616B65202120424C444F31206D617825
:208EA000696D756D206F757470757420766F6C74616765206973202025756D56004D697355
:208EC00074616B65202120444C444F31206D696E696D756D206F757470757420766F6C7466
:208EE000616765206973202025756D56004D697374616B65202120444C444F31206D6178C3
:208F0000696D756D206F757470757420766F6C74616765206973202025756D56004D6973F4
:208F200074616B65202120427574746F6E2062617474657279206368617267696E6720739E
:208F400074657020766F6C74616765206973202575206D56004D697374616B65202120549A
:208F60006865206D696E696D756D20636861726765207465726D696E6174696F6E20766FAF
:208F80006C74616765206F662074686520636F696E2063656C6C2062617474657279206941
:208FA00073202575206D56004661696C656420746F207365742074686520706F776572201F
:208FC0006368616E6E656C2C2074686520706F776572206368616E6E656C20686173206207
:208FE00065656E2070726F746563746564004D697374616B65202120444331206D696E699B
:209000006D756D20766F6C74616765206973202575206D56004D697374616B6520212044E3
:209020004331206D6178696D756D20766F6C74616765206973202575206D56004D69737456
:20904000616B65202120414C444F31206D696E696D756D206F757470757420766F6C7461FA
:209060006765206973202025756D56004D697374616B65202120414C444F31206D6178693C
:209080006D756D206F757470757420766F6C74616765206973202025756D56004D69737468
:2090A000616B65202120414C444F32206D696E696D756D206F757470757420766F6C746199
:2090C0006765206973202025756D56004D697374616B65202120414C444F32206D617869DB
:2090E0006D756D206F757470757420766F6C74616765206973202025756D56004D69737408
:20910000616B65202120414C444F33206D696E696D756D206F757470757420766F6C746137
:209120006765206973202025756D56004D697374616B65202120414C444F33206D61786979
:209140006D756D206F757470757420766F6C74616765206973202025756D56004D697374A7
:20916000616B65202120414C444F34206D696E696D756D206F757470757420766F6C7461D6
:209180006765206973202025756D56004D697374616B65202120414C444F34206D61786918
:2091A0006D756D206F757470757420766F6C74616765206973202025756D56004D69737447
:2091C000616B652021204350554C444F206D696E696D756D206F757470757420766F6C7464
:2091E000616765206973202025756D56004D697374616B652021204350554C444F206D61C5
:2092000078696D756D206F757470757420766F6C74616765206973202025756D5600504D05
:2092200055206973206E6F74206F6E6C696E652E2E2E0067657449443A307825780A00598E
:209240004553004E4F0069734368617267696E673A0069734469736368617267653A006997
:20926000735374616E6462793A00697356627573496E3A00697356627573476F6F643A00C0
:20928000676574436861726765725374617475733A007472695F63686172676500707265B5
:2092A0005F63686172676500636F6E7374616E742063686172676500636F6E7374616E7487
:2092C00020766F6C746167650063686172676520646F6E65006E6F74206368617267696EFF
:2092E0000067657442617474566F6C746167653A0067657456627573566F6C746167653AAB
:209300000067657453797374656D566F6C746167653A00676574426174746572795065723A
:2093200063656E743A002500535441545553203D3E204845583A002042494E3A0069734413
:20934000726F705761726E696E674C6576656C3200697357647454696D656F7574006973EE
:209360004261744368617267654F76657254656D7065726174757265006973426174576FA9
:20938000726B4F76657254656D7065726174757265006973426174576F726B556E64657232
:2093A00054656D706572617475726500697356627573496E73657274006973566275735260
:2093C000656D6F7665006973426174496E7365727400697342617452656D6F7665006973CC
:2093E00050656B657953686F72745072657373005265616420706D752064617461206275B3
:2094000066666572202E002C00697350656B65794C6F6E67507265737300697350656B6557
:20942000794E6567617469766500697350656B6579506F7369746976650069734C646F4F09
:2094400076657243757272656E744972710069734261746665744F76657243757272656E73
:2094600074497271006973426174436861676572446F6E650069734261744368616765724C
:2094800053746172740069734261744469654F76657254656D7065726174757265006973B3
:2094A0004368616765724F76657254696D656F75740069734261744F766572566F6C74614A
:2094C0006765000D0A00232D302B2000686C4C0065666745464700303132333435363738E6
:2094E00039414243444546003031323334353637383961626364656600000000000000003C
:2095000000000000E7070008470A00084907000857070008050800081902000839020008C3
:209520005D0300085D010008B51100087D100008210A00086F080008190800084D110008B9
:20954000F112000879070008FF08000831190008793100088731000897310008313100086B
:20956000691E00086B150008EF080008831E0008F9110008C908000837150008B908000824
:2095800003150008A30800082D080008C31100089514000889140008B3010008C9010008FB
:2095A000870100089D0100085F01000871010008DF010008F5010008F9100008E31200089F
:2095C00007110008D512000823110008C71200083F110008B912000815110008AB12000841
:2095E000311100089D12000819100008D31400088D080008A11400087D0800080000020061
:2096000000050000030000043029003928005D7D005B7B00B70000B5D600B6D700B4000051
:20962000859000848900838800828700818600607E00332300324000080000D4D500C100D5
:209640000009D200B1D0003424004500005700005000003D2B002D5F005C7C002F3F0052DE
:2096600000005300003121000AD100382A00372600365E00352500460000580000510000CE
:209680002E3E004900005500005900005400005600003B3A004100004C00004B00004A0026
:2096A000004800004700004300002722005A00004F00002C3C004D00004E0000420000445D
:2096C0000000200000000000C8C91213141516171C1D1E1FCACBCCCDCECF2627C0C1C2C3CA
:2096E000C4C5C6000000000000000000EF28000831290008DD2500088D2A0008E1250008C3
:20970000E925000803260008AB7C0008CD7C0008010202030405060708090A0B0C0D0E0F08
:2097200010100201040302040810040040000004010100000202000004040000080800007B
:209740001010000020200000404000008080000001000104020002040400040408000804FB
:209760001000100420002004400040048000800400000000010203040000000000000000EF
:2097800001020304060708090000000000440040120000000B000000003801401200000075
:2097A0001D00000000480040120B00001D01000000480040120A0000FFFFFFFF0000000029
:2097C000000000000100000000440040120800000C00000000380140120000001E00000035
:2097E00000480040120000001E01000000480040120A0000FFFFFFFF000000000000000010
:209800000300000000440040100800000A0000000038014010060000170000000038014080
:20982000100500001B00000000480040100000002B00000000480040100A0000FFFFFFFF97
:209840000000000000000000020000000044004012080000090000000038014012060000CE
:209860001600000000380140120500001A00000000480040120000002A00000000480040DC
:20988000120A0000FFFFFFFF000000000000000000000000000000401280000000010000DD
:2098A0000000004012900000010000000000004012120100010100000000004012100100FB
:2098C000020000000000004012920100020100000000004012910100030000000000004077
:2098E0001212020003010000000000401211020006000000000400401295000007000000E1
:20990000002C0140128D100007010000000400401215010008000000002C0140128E0000A2
:2099200008010000002C0140128D000009000000002C0140120E010009010000002C014004
:20994000120D01000A000000002C0140128E01000A010000002C0140128D01000B000000AC
:20996000002C0140120E02000B010000002C0140120D02000F0000000000004012910000CC
:209980000F01000000000040128F000010000000002C0140120D11001001000000040040D4
:2099A0001295010010020000000400401294010011000000002C0140128D110011010000C2
:2099C000000400401215020011020000000400401214020013000000000000401211010024
:2099E0001301000000000040120F010014000000000400401294000015000000000400409A
:209A0000121401001600000000080040129700001700000000080040121701001800000077
:209A200000080040129701001900000000080040121702001A0000000000004012900100AB
:209A40001A01000000000040128F01001B00000000000040121002001B010000000000402E
:209A6000120F02001D000000002C0140128E10001E000000002C0140120E11001F000000AE
:209A8000002C0140128E110026000000000400401293000027000000000400401213010008
:209AA000280000000004004012930100290000000004004012130200FFFFFFFF0000000004
:209AC0000000000016000000005400400A04000018000000005400400A0300001A000000FB
:209AE000005800400A000000FFFFFFFF000000000000000017000000005400400A0400000F
:209B000019000000005400400A0300001B000000005800400A000000FFFFFFFF00000000D2
:209B2000000000000000000001000000020000000300000004000000050000000600000010
:209B4000070000001000000011000000200000002100000022000000230000002400000033
:209B60002500000000000000010000000200000003000000040000000500000006000000AB
:209B80000700000008000000090000000A0000000B0000000C0000000D0000000E00000071
:209BA0000F0000001000000011000000120000001300000014000000150000001600000011
:209BC0001700000018000000190000001A0000001B0000001C0000001D0000001E000000B1
:209BE0001F0000002000000021000000220000002300000024000000250000002600000051
:209C00002700000028000000290000002A0000002B0000002C0000002D0000002E000000F0
:209C20002F000000300000003100000032000000060007000800000000000000000000004D
:209C400005760008B5760008E975000813790008BF750008F97A0008CF750008AB7C000822
:209C6000CD7C0008A864FF7F01000000117E00084101000859200008212C00085968000888
:209C8000297B00081D010008B1200008312C0008316900081428506EFF0100001000000008
:209CA00000080140000C0140001001400014014000180140003002400000000000127A0011
:209CC000000000000000000000000000000000000000000000000000000000000000000084
:209CE000000000000000000000000000000000000000000000000000000000000000000064
:209D00000000000000000000000000000000000000000000FFFFFFFFFFFFFFFFFFFFFFFF4F
:209D2000FFFFFFFF0003000000000000000000000000000000000000000000006809002093
:209D4000E80300000800000008000000BC000020000000002808002090080020F808002004
:209D60000000000000000000000000000000000000000000000000000000000000000000E3
:209D800000000000000000000000000000000000000000000000000000000000FFFFFFFFC7
:209DA000FFFFFFFFFFFFFFFFFFFFFFFFFFFFFFFFFFFFFFFFFFFFFFFFFFFFFFFFFFFFFFFFC3
:209DC000FFFFFFFFFFFFFFFFFFFFFFFFFFFFFFFFFFFFFFFFFFFFFFFFFFFFFFFFFFFFFFFFA3
:209DE000FFFFFFFFFFFFFFFFFFFFFFFFFFFFFFFFFFFFFFFFFFFFFFFFFFFFFFFFFFFFFFFF83
:209E0000FFFFFFFFFFFFFFFFFFFFFFFFFFFFFFFFFFFFFFFFFFFFFFFFFFFFFFFFFFFFFFFF62
:00000001FF
